:020000020000FC
:02000000B5C188
:02000800020EE6
:100034000C94692B0C94672B0C941C1D0C94351E8A
:1000440046E00895D5C1DBC1E5C1E9C1C8EDD1E001
:100054000895C4E1D1E00895C0E0D1E00895CCE36F
:10006400DDE00895E0E0F6EF0895E0E0F6EF0895AE
:10007400C8E8D1E00895CEE2DDE00895C8E7D1E014
:100084000895C0EADCE00895C0EFD0E10895FF913F
:10009400FF93EF2FE854F2E4FA5FE650E8F7EE2717
:1000A40026F4EA0FFB1FEE0FFF1F08956894EFCFAD
:1000B400E894EDCFFF91FF93E0E0F854F65010F090
:1000C400E395FCCF08950C9487330C94AC330C94D3
:1000D400B8330C9423330C949C330C94BA380C949A
:1000E400A63B0C94A03B0C9496330C9499330C943B
:1000F4004B340C94DF340C94DB330C9436340C9472
:1001040097360C9476360C947E36E8940C94D0375B
:1001140068940C94D0370C940F3F0C949D340C9439
:100124003B3E0E9497360C94F5380C94E6380C94B8
:10013400EE38409120014F7108954091390108959E
:100144004091220108954091230108954091210195
:1001540008950C94443A0C945D3A0C94AF3A0C9480
:10016400503A0C946D3A0C94C63A0C946F390C9432
:10017400BD3F0C94973F0C94303A0C94393A0C944C
:10018400773A0C941D3A0C94B3360C9492380C9430
:1001940017380C9430380E94D3180C942D3D0E94CB
:1001A400D3180C94623D0C94183D0C941F3D0C9490
:1001B400263D0C94D43A0C941F3B0C94B03D0C9403
:1001C400F33D0C94AB3D0C94EE3D0C94BA3D0C9471
:1001D400FD3D0C94B53D0C94F83D0C9443380C94BF
:1001E4006F380C943C250C945E250C94C2380C9406
:1001F4008F3B0C94D03F0C94EC3F0C94F03F0C9448
:1002040030400C9443400C94FE3F0C94FA3F0C9401
:1002140004400C9409400C9400400C944E400C94FF
:1002240070400C9479400C940B0D0C94240D0C9498
:10023400230D0C942F0D0C948D0D0C94580D0C94CF
:100244005B0D0C94AE0D0C94B50D0C94BD0D0C947B
:10025400CE0D0C94DE0D0C945F0E0C947A0F0E945C
:10026400C4420C9403260E94C4420C940C260E949F
:10027400C4420C9415260E94C4420C941E260C946D
:1002840063420C94B0400C9445420E9425430C9464
:10029400074188270C94392688270C9444260C940B
:1002A4002F0E0C943A0F0C94A2250C94A6250C94B2
:1002B40076230C94BE3B0C94AA3B0C9453100C94E0
:1002C400610B0C940A1E0C94A81B0C94B91B0C947F
:1002D400C2280C9485280C94F0780C949A200C94E1
:1002E400FA790C94257A0C94A2180C94F8180F90AF
:1002F4000F900C94462D83D00C947234AF93BF931B
:100304000C9423350C94AB360C94C336AF93BF9343
:100314000C94A9340C94D61E0C94F91E0C948539B3
:100324000C94B31C0C94D91CA093FF100895A091B5
:10033400FF1008950C949A0F0C9495400C949B40D4
:100344000C948F40E3E109C0E5E107C0E4E105C096
:10035400E6E103C0E7E101C0E8E1F091F410F7FF42
:1003640009940F900F900895F894A0E02A2EA1E02C
:100374003A2EA0E1AEBFAFEEADBF2092FF100E94B7
:100384009B320E94F33F0E9476780E9476780E9406
:100394002B3B0E94FA79F091F010FFEFE8E1F7FFB0
:1003A400099520924A01AA270E9423330E944B34C4
:1003B400AFEFA0931001A0933D0120924901209238
:1003C4005C018827209239012092220178940C94B0
:1003D400200242954A9540934901A7E00E94873341
:1003E400AA270E94B8330E944B340E94E804BCCF71
:1003F400AF91BF91CF91DF91EF91FF9108950F904D
:100404001F90FF93EF93DF93CF93BF93AF931F920C
:100414000F9208957F916F915F914F91E9CF0F9063
:100424001F90FF93EF93DF93CF93BF93AF934F93BB
:100434005F936F937F931F920F920895A1E00E94A0
:10044400B8339927A0E10E9487330E944B34C4E05B
:10045400DAE0E7E3F7E10E943038A7E00E9487334F
:100464000E947E360704200005D1A6E10E9487334E
:1004740006D1C5E0D8E0E6E0F9E00E943038D8E1E2
:10048400F9E10E943038D8E0F9E0CC5FEC5FC83382
:10049400A0F364EB0E94BA384091200141FD19C0D9
:1004A40040912301403011F00C948A026A9591F72F
:1004B400ECE0F0E958E044914C3421F4E0E1F695A5
:1004C400099503C0F45F5A95B1F74AB5407761F3D3
:1004D40080CF0E944B340E947E3600004B657962C7
:1004E4006F6172642D54657374000E949D34709121
:1004F4007101A0917101A215E1F32092710190E0C4
:100504007A2F0E9436340E94DE34F3CF0E94EE38F4
:10051400A0E00E94B833A1E00E94263A99272092D5
:100524003601AA270E942333A5E00E9487330E9444
:100534004B34C0E0D0E0EDE1F5E10E946F38C2E158
:10054400D4E0A8EFA993A1EFBCE1A993BA95E9F788
:10055400A9EFA993A1E50E948733A4E0B1E00E942A
:10056400973688D02CD1409149014B3008F044276C
:1005740040934901642F67FD66276B3008F06AE0F9
:1005840020E06F938CD06F9123952830D1F76DD1F3
:1005940049D1F2D0E0E5FAE00E94D43A423E11F4A7
:1005A4006A95E9CF433E11F46395E5CF443E21F4C7
:1005B400643010F06450DFCF453E21F4673010F40E
:1005C4006C5FD9CF4A3E11F04530E1F4683088F0D1
:1005D40029F40E94EE380E941E2198CF693021F43C
:1005E40059D00E94552692CF0E94EE380E94DF27F0
:1005F4008DCF4ED088270E94E8040E9476780E940E
:100604002B3B84CF683030F6423029F441D0882720
:100614000E94CB047BCF433021F43AD00E94A7221E
:1006240075CF443031F434D00E9400230E94DB0A99
:100634006DCF473021F42CD00E945A0467CF483044
:1006440031F426D00E945E250E9483285FCF493072
:1006540041F41ED00E945E250E94C0280E94DB0A3D
:1006640055CF4A3031F414D00E94A4040E94DB0A0E
:100674004DCF90CFE0E8FFE80E9476360895A0E0E1
:10068400B7E10E949736E6E9FFE80E9476360895BE
:1006940060934901A0912201A030E1F70895A1E0FF
:1006A400B3E020FDA95F21FDA25F22FDBA5F422FC6
:1006B4000E943079423439F4E8944EE004910F35C5
:1006C40041F44CE006C0452F440F44FB4E7040F902
:1006D4006894621709F44295409338010E94973652
:1006E4001EF10E947E36FF20200040E50E94DF3488
:1006F400422F4F5C0E94DF340E947E36FF20200090
:10070400B3950E9497360E947E36FF2020D0D120D8
:100714002000B3950E9497360E947E36FF2020D297
:10072400D3202000B39513C070960E94973613E02F
:1007340004E00E94DE3445910E94DF340A95D9F723
:100744000E94DE34B3950E9497361A9589F7422F9A
:100754000E94AC790E94973666E045910E94DF348E
:100764006A95D9F7B3950E94973666E045910E9441
:10077400DF346A95D9F708954AE06A3009F442955E
:10078400409338010E947E360F0F20202020202025
:1007940000000E947E36100F2020D4D520200000B7
:1007A4000E947E36110F2020D6D7202000000E9400
:1007B4007E36120F20494E464F20000008954AE02D
:1007C400409338010E947E3614024D43553A363424
:1007D400340040E2F29940E50E94DF340E947E3604
:1007E40014164B42443A0000E0E0F9E844910E94B8
:1007F400DF34E05844910E94DF340E947E36140CAA
:100804005649443A00007BB572FD06C00E947E360C
:10081400FF4E5453430005C00E947E36FF50414CA6
:100824002000089548E0693009F442954093380166
:100834000E947E360F0820202020202000000E94E5
:100844007E3610082020D8D9202000000E947E3651
:1008540011082020DADB202000000E947E361208D6
:10086400434F4E464947000008954CE0683009F470
:100874004295409338010E947E360F0120202020AB
:10088400202000000E947E3610012020DCDD202084
:1008940000000E947E3611012020DEDF20200000AF
:1008A4000E947E36120144464C415348000008958C
:1008B400A4E00E948733C1E0DEE0ECE1F2E10E94B3
:1008C4006F38A0E40E9487330E94DB0A0E947E36C0
:1008D4000F02436F70792050726F6772616D2074DC
:1008E4006F007091490160E0ACE0671709F4A0E67D
:1008F4000E948733B1E1A62FAA0FA60FAD5F0E9415
:10090400973640E50E94DF34462F47704F5C0E94C3
:10091400DF346395683041F70E94E638423E21F4A3
:100924007030D1F37A95DFCF433E21F47730A1F3D1
:100934007395D9CF4A3E19F40E94D77908954D3E54
:1009440059F70895AFE20E948733C1E0DEE0ECE19D
:10095400F2E10E9443380E94DB0A0E947E361002B4
:10096400436C65617220746869732070726F67727A
:10097400616D2028792F6E293F000E94E63849379F
:1009840029F04E3629F04D3E19F0F7CF0E94B57983
:1009940008950E94EE380E942E794E3451F04C3462
:1009A40041F00E94A80520923901A0912301A43F9F
:1009B40009F0AECD0E942E7944914F3551F306D003
:1009C4000E942B3BAA270E942333E3CF0E944B347F
:1009D4000E94FA798827209222010E94AA794491E0
:1009E4004F3571F03C964591423459F04E3441F400
:1009F400459144FD0895F695E0E109950E942B3B4D
:100A040008950E94EC0F0E942B3B20921901209222
:100A14005C01ABB5AF77ABBD209236010E94A63B1B
:100A240083FCAEEE83FEA4E4A0931B01A0913901E4
:100A3400A1FD07C0A0912201AD3E91F70E94EE38BE
:100A4400089520921B010E948539EACF202020209E
:100A54002020204564697420205361766520204C51
:100A64006F6164202052756E202003002020202016
:100A7400202020436F7079202053656E642020521B
:100A84006563762020436C656172A0E00E94B833F0
:100A9400A3E00E94263A8F93409149010E94A578D1
:100AA4000E944B340E941A3399274091220140300E
:100AB400E1F70E947E3600002050524F4752414DCC
:100AC4002000409149014F5C0E94DF344AE30E94B8
:100AD400DF34C3EED1E02FD2CFD20E947979CBD3C9
:100AE4008F91A8E8803069F1ACECEAEAF2E1813058
:100AF40031F0ABE48A9545914030E9F7F8CF23D241
:100B040092E0A5E0B1E00E9497360E9476360E94FA
:100B14007E36FF20494E20500000409146014F5C34
:100B24000E94DF344AE30E94DF34BB27AC2DA39537
:100B34000E94DB334AE30E94DF34AD2DA3950E946B
:100B4400DB330895AAE25A2E70E208959927FADF5A
:100B54009CDF1AD5D0923A010E940E390E94853941
:100B640050912001403E21F4AA2752FDBB2733C0F7
:100B7400413E31F4AFE152FDAA2752FDBEE52BC040
:100B8400423E11F4AA9527C0433E69F4A3959B2FD6
:100B94000E94B40A9A1730F4BE3511F4AA951BC00A
:100BA400AA27B39518C0443E21F4BA95B7FDBB27D4
:100BB40012C0463E21F4B850B7FDBB270CC0473ED7
:100BC40011F4B85F08C0453E11F4B39504C04A3E21
:100BD40039F5B395AA27A03838F0AFE1BA95B03803
:100BE400C0F0AA27BB27B6CFA03228F0BE3589F0C3
:100BF400AA27B395AFCFBF3508F0BEE50B2F0D156F
:100C040008F4D02E0D2D015F0B1718F40B2F0F5085
:100C1400D02E9B2F0E94B40A9A1708F4A92F9ACFBA
:100C24009B2F4E3E39F4AF93BF930E94800ABF912D
:100C3400AF9159C14F3E31F4BF930E948B0ABF91CB
:100C4400AA2751C1493E11F463D14DC14C3E31F440
:100C5400A03009F481CFAA955BD145C1547009F441
:100C64009CC0433FD9F4ACEC6ED10E947E360107A0
:100C7400524543454956452050524F4752414D2015
:100C8400592F4E203F0050D136F447D2F4D25ADFC8
:100C940090D45092D8014FD188275BCF423FE1F4E2
:100CA400ACEC51D10E947E36010753454E4420508E
:100CB400524F4752414D20592F4E203F000034D10E
:100CC40056F7ACEC40D10E947E36010753454E44A2
:100CD400494E4700A1E038C0443FC1F4ACEC33D1E5
:100CE4000E947E360107434C4541522050524F47E3
:100CF40052414D20592F4E203F0016D136F4ADD22B
:100D0400BAD220DF56D45092D801C5CF413F19F54D
:100D1400ACEC19D10E947E3601075052494E542042
:100D240050524F4752414D20592F4E203F00FCD086
:100D34008EF4ABE408D10E947E3601075052494E2E
:100D440054494E470000A2E0A093360131D12092CD
:100D54003601F8DEA0CF433611F44AD2FDCE48372F
:100D640031F40E94FA0869D25092D80110C0C5EF3C
:100D7400D1E0463771F46881623451F466E0299217
:100D84006A95E9F72AD277D25092D801E5CE88271E
:100D9400E3CE4636E1F724D4DFCE423F11F5BF93CC
:100DA400AF93C5D0D9F0ACECCED00E947E3601070B
:100DB400534156452050524F4752414D20592F4ED2
:100DC400203F0000B1D046F40E943C790E9479791A
:100DD40052D2B8DE7093D801AED08827AF91BF91BC
:100DE400B9CE433FE1F4BF93AF93A1D0B9F0ACECDB
:100DF400AAD00E947E3601074C4F535420434841E9
:100E04004E47455320592F4E203F00008DD026F7E2
:100E14000E94797930D296DE7093D801DDCF413FBC
:100E240039F43D01AAD0D3015092D80195CED4CF44
:100E34004D3E11F5BF93AF937AD0A9F0ACEC83D0BB
:100E44000E947E3601075155495420572F4F205395
:100E540041564520592F4E203F0066D046F7A091B9
:100E64002201A030E1F70E941533A0E00E94233351
:100E7400AF91BF91A1D30895443FE9F49DD357D0D6
:100E840029F40E9415330E944B340895A9E65BD0DF
:100E94000E947E36010753415645204348414E4740
:100EA4004553204245464F52452052554E2100009D
:100EB4000E94E63891CF4B3E59F4A93148F440E200
:100EC40015D040E2EA2FE35071F0E8F70FD0F9CFE4
:100ED4005091200152FD09C053FD07C04C3128F048
:100EE400403818F403D05092D80136CEAF3161F0B7
:100EF4005A2FAFE10E9466396A916983AA95A517B2
:100F0400D9F74883A39508950E94663948830895C4
:100F14000E9466395A2F5F3121F0498149935395D4
:100F2400FACF50E2588308950E94FF3D0895A0919E
:100F3400D801A0320895A8E806D00E947E360105A3
:100F44004F4B00000895EF93FF939927A0934C0112
:100F54000E947E36010520202020202020202020F1
:100F6400202020202020202020202020202020207D
:100F740020202000FF91EF910895A0E00E943639CF
:100F84004A3E09F40895423E21F4A030B9F3AA95EB
:100F9400F5CF433E21F4AB3089F3A395EFCF403234
:100FA40068F3403858F74883AB3009F0A395E6CF8F
:100FB400C9EDD1E057E049910E94DF345A95D9F741
:100FC40056E122965DE049910E94DF345A95D9F7A3
:100FD4000E949D344EE511D016F04A95E1F7542F46
:100FE40053954427451719F024D04395FBCF43E28A
:100FF4000E94DF340E949D340895CF93DF935F9362
:101004006F93E894C4E4D2E053E2459FC00DD11D30
:1010140050E26991613238F45A95D9F76F915F9132
:10102400DF91CF91089568946F915F91DF91CF9193
:101034000895DF93CF934F935F936F93C1E4D2E00E
:1010440053E2459FC00DD11DDF93CF93A39653E286
:101054006A91613210F45A95D9F7CF91DF91499191
:101064000E94DF345A95D9F70E949D346F915F91A5
:101074004F91CF91DF9108950E9401024F93EAE9C5
:10108400F0E1AEE1B2E04591403011F04D93FBCF79
:101094004F910C94FA0120457869742020204E6108
:1010A4006D6520202053617665202052656C6F6148
:1010B4006420202052756E2020000E9401024F936C
:1010C400EAECF0E1DECF2020202020202020507206
:1010D400696E74202053656E642020205265637607
:1010E400202020204E65772020000E9401024F938B
:1010F400EAEFF0E1C6CF2041626F72742020202015
:1011040020202020202020202020202020202020DB
:1011140020202020202020202000E7DFACEC13DF5B
:101124000E947E360105524543454956494E472E95
:101134002E2E000020923A0190D09DD09927ECECFD
:10114400E0934C01E3EEF1E0EE2EFF2E41E10E942C
:10115400423A5CE00E94AD3A4B31B9F14A33D1F7DF
:101164000E94AD3A4B3189F1403218F041935A95BF
:10117400B9F7403228F00E94AD3A4B3131F1F9CF42
:10118400EEE1F2E0EE2EFF2E53E2EE2DFF2DB396AC
:10119400EE2EFF2E0E94AD3A4B31B9F04032D0F31F
:1011A400433299F006C00E94AD3A4B3171F040329F
:1011B40048F041935A95B9F70E94AD3A4B3129F062
:1011C4004032D0F793959036F9F60895A3E2BA9F8A
:1011D400A1E4B2E0A00DB11D08953D01F7DFC8E818
:1011E400D1E053E249914D935A95E1F7D301089523
:1011F4003D01C5EFD1E0A2E4A993A5E5A993A6E436
:10120400A993ADE3A993E2DFC8E8D1E053E24D919D
:1012140049935A95E1F7C5EFD1E0A2E4A993A5E576
:10122400A993A6E4A993ADE3A993409188014993B6
:10123400409189014993D3010895BF93AF934F938C
:101244005F93C4DF139640E250E24D935A95E9F759
:101254005F914F91AF91BF9108950E9401024F9306
:1012640040E2A1E4B2E0CDEFDCE04D932197E9F751
:101274004F910C94FA010E9401024F9341E0A1E4C2
:10128400B2E0C0E3D42FDA5010F0C395FCCFD65CA3
:10129400CD93DD93C0E2CD9390964395403689F784
:1012A4004F910C94FA01425245414B004F5645521E
:1012B400464C4F5700444956494445202F3000536B
:1012C40051522046524F4D203C3000434F4E535410
:1012D400414E5420544F4F204249470057524F4EDD
:1012E400472045585052455353494F4E0053594E89
:1012F400544158204552524F5200554E4B4E4F5771
:101304004E204B4559574F52440057524F4E472099
:10131400464F524D415400424144204C494E454EA3
:10132400554D424552004E45585420572F4F2046A4
:101334004F520052455455524E20572F4F20474F7D
:1013440053554200535441434B204F564552464C4B
:101354004F5700554E54494C20572F4F205245505B
:1013640045415400493243204552524F5200554E94
:101374004B4E4F574E204552524F520044464C411B
:101384005348204552524F52004F5554204F462047
:10139400415252415900494E434F4D504C455445DA
:1013A40020504152004B4559574F52442049532035
:1013B4004D495353494E470057524F4E47204243DD
:1013C4004F505920004F5554204F46205343524507
:1013D400454E0043414E4E4F5420435245415445DF
:1013E4002046494C45004D454D4F52592046554CD9
:1013F4004C0046494C45204E4F5420464F554E44D0
:101404000050414745204E4F5420494E2046494CF8
:1014140045005041474553204E4F5420494E2052D9
:10142400414E4745004E4F5420494E2047524150AB
:1014340048494353204D4F4445004E4F5420494E94
:101444002054455854204D4F4445004E4F20555389
:10145400522046494C4500535243204F5554204F87
:10146400462053435245454E0044455354204F555E
:1014740054204F462053435245454E0057524F4E39
:1014840047205350524954450057524F4E47204528
:101494004550524F4D20414452004E4F2050524728
:1014A4002046494C4500584D4F44454D2045525225
:1014B4004F520043414E54204C4F4144205448491C
:1014C4005300494F2044495341424C45440053453D
:1014D4005249414C31204E4F5420415641494C41D0
:1014E400424C45004E4F20494F20445249564552E4
:1014F400004E4F204C49425241525900BE3508F02B
:101504000895BF9323D0B395BE35E1F796DEBF911E
:10151400B2CEBE3508F00895BF93AF93AB2FAA9512
:10152400BDE508D0BA95BA17E1F7B39586DEAF9159
:10153400BF91A1CE0E94010249DE1396ED01B0E2F3
:10154400A991AAA3BA95E1F70C94FA010E940102A9
:101554003DDE1396ED01B0E2ABA1A993BA95E1F794
:101564000C94FA010E94010231DEED0193964E9132
:101574004132E8F34038D8F7AC1BBC0B9A2F925099
:1015840097FD99270C94FA0122D00E9470404F35A0
:1015940020F0AA27BB27D22C0895B42F0E947040B4
:1015A4004032B8F7A42F0E947040403590F7D42EF3
:1015B4000895AA27BB27D22C0AD04B2F0E9479402A
:1015C4004A2F0E9479404D2D0E9479400895009041
:1015D4004901C0EDD7E043E0409DC00DD11D089501
:1015E4003D01AEE2B0DC0E947E36010546494E4420
:1015F4003A00E0E0F0E8C0E0D2E0CE0FF8830E94C9
:10160400E6384D3E89F04A3E91F04C3E29F4E030F4
:1016140091F32882EA95EFCF403868F74883E39541
:10162400E03149F7EA95E7CF86DCD3010895E0304D
:10163400D9F3F72D03E20F9FA4E4B2E0A00DB11D8E
:1016440010E2C0E01E1730F14E2E222709901D90A3
:1016540023950114D1F44A94C9F725D07F2E00E2D2
:10166400011B602E072D085008F400270F3408F0E2
:101674000FE400933A010E94E6384A3E29F04D3EB9
:1016840089F7D02E10D0D0CF0ED01A95A21BB20954
:101694001196D7CFF395FF3509F4FF274091220126
:1016A4004D3E41F6C1CF0E94EE38AE1BB2094E2E1C
:1016B4000C9100580D934A94D9F708952DC1CAEF9F
:1016C400DCE02A922A9280E02F92AA27BB274427A3
:1016D40071917032E9F3703888F77A3379F3BB2764
:1016E4007E3709F038C07191733511F4D40138C0D4
:1016F4007C3419F4AC2DA39533C0703521F4A0913A
:101704004601A3952DC0763531F4BBB5A9E3B2FFEC
:10171400A7E0B1E025C0783519F4A091500120C0AC
:10172400793519F4A09151011BC0723529F4A091A7
:101734002E0DB0912F0D14C07E3419F4A0913A0DE2
:101744000FC07D3421F4A1E0F299A2E009C07832FF
:10175400D1F47CE10FC07C3111F07E3119F4A191F8
:1017640071911EC07D3111F07F3111F4B191F7CF29
:101774007C3158F4572F2E01EF015F93452FAA2790
:10178400FE01E201A5CF87E0D7C07033B0F07A3311
:10179400A0F4403810F086E0CFC0A72FA053719179
:1017A400703211F47191FCCF4F3709F434D1AA93FC
:1017B400BA9340E890CF85E0BFC07134A0F07B3588
:1017C40090F4403810F086E0B7C07154770FEF936F
:1017D400FF93E0EAFCE0E70FF21DA191B191FF91C4
:1017E400EF917191DDCF7D3251F44F3711F44427DD
:1017F4006FCF20F4403210F04FE76ACF59C07832EF
:1018040031F471E07F93AA27BB27472F61CF793248
:1018140009F048C05F915D3188F5B991A991FF93B2
:10182400EF93DF93CF9306E40F930CE00F9300E262
:101834001CE0050F121D0F931F93089586E0089571
:10184400E8C0F7C0A6C117C0B7C137C26BC289C20E
:10185400A4C2ABC2A9C2ABC28EC2FAC2E2C126C143
:1018640028C1E6C1FAC1B3C1BAC1BFC13AC249C2B3
:10187400FFC23EC34EC3B095A095089574D0803086
:1018840009F05AC0C7CF86E00000CF91DF91EF91F5
:10189400FF91803009F050C0AA93BA93AA27BB27BE
:1018A40042E016CF4F3720F44F3110F086E044C0A9
:1018B400608132E27C3359F46E3341F033E26D33AC
:1018C400F9F13EE46C33E1F131E23BC039C07E33DF
:1018D40041F435E26D33A1F13FE46E3389F134E232
:1018E40030C036E27D3369F137E37B3251F138E3BE
:1018F4007D3239F139E5733221F130E37E3509F176
:101904003AE57A32F1F03BE57F32D9F03CE57532C5
:10191400C1F03DE37632A9F05F91503021F05F31A0
:1019240030F021D0F9CFB991A9913197089586E08B
:101934005F915030C1F3FCCF4F914030E9F70895E7
:101944003196732F5F91A72FB52FA07FB07FBA1761
:1019540020F009D0803081F7F5CF5F937F93AA27D9
:10196400BB27472FB5CE5F934F9319910991B99136
:10197400A99126EC352F3F70330F330F230F3CE032
:10198400321D2F933F930895A027B1273DC0000037
:10199400EAD03AC000000000DFD0A150A17034C0EA
:1019A400EAD0A150A17030C0E6D02EC000000000E3
:1019B400DAD0A150A17028C0CFD026C0000000000A
:1019C40041D022C0000000003CD01EC00000000036
:1019D400A02BB12B19C0000040D016C0000000009D
:1019E4009AD012C00000000096D0A22FB32F0CC0D2
:1019F400A023B12309C00000DDD206C0000000000E
:101A0400E1D202C000000000AA93BA934F915F9103
:101A14000895B7FF0895A095B09511960895AA93D7
:101A2400BA93089517FF089500951095030D121D9C
:101A34000895AB2B29F0B7FBA1E0BB270EF4129756
:101A44000895F2DF2B2F2127A00FB11F27FD089542
:101A54002B2F212727FD82E008950BD0D901BF77D2
:101A64000EF4D9DF37FD03C0452B09F4089582E055
:101A740008956DD0CEDFB19FA001A09F9001A19FDA
:101A8400300D411D521DB09F300D411D521D089552
:101A940008E611E0B03818F0A00FB11FFBCFA01773
:101AA400B10718F0A01BB10BFACF08950AE5A01BEB
:101AB400B209EEDFE4EAF7E80AE510E0A017B1079F
:101AC40038F4E00FF11FEA1BFB0BA491BB27089528
:101AD40004EB10E0A017B10768F40AE510E0E01B7E
:101AE400F10BEA0FFB1FA491BB27A095B095A30DA2
:101AF400B21D08950EE011E0A017B10728F4E00F1D
:101B0400F11FEA1BFB0BEFCF0EE011E0E01BF10B22
:101B1400EA0FFB1FDACF212F202B11F483E0089565
:101B240016D022273327442751E1441FAA1FBB1F85
:101B34005A9551F0221F331F4FEF201B310BA8F78A
:101B4400200F311F40E0F1CF0EF465CF08952B2F05
:101B5400212727FB5EDF66CF0F931F930A271B27DE
:101B6400012B91F00FC00F931F93B0581058A01B76
:101B7400B10B50F007C00F931F93B05810580A1BB5
:101B84001B0B10F0AA2701C0A1E0B0E01F910F9138
:101B9400089584E0B7FD089588270A2F1B2FB2E02B
:101BA400AA27232D3327021B130B20F0A3952B0FF9
:101BB400321DF9CFBB2708954F935F938D010E9487
:101BC4003F3B59DFA42FB52F5F914F910895AF3F4D
:101BD40011F0A0933F01A0913F01BB270895AEBD32
:101BE4000E94AF1CAEB5BB27089510914A01103076
:101BF40011F08CE10895AA95AE3510F08AE00895AD
:101C0400E0E0F0E9B0E2AB9FE00DF11DA0914601E8
:101C1400BCE0AB9FF00DB1960E94D43AA42FBB2731
:101C24000895B0937301A09372010E94B51C0895A6
:101C3400BF3F69F0A09378010E94D425803021F041
:101C4400AFEFBFEF88270895A42FBB2708950E9404
:101C5400F1258827B42FAA270895BF3FA1F4A0FD3A
:101C640009C00E94E825803019F08827CC27DD2799
:101C7400DE0108950E94E825803019F08827EE27B8
:101C8400FF27DF01F6CFA09378010E94D42580308E
:101C940021F08827AA27BB27ECCF7F9377270E94C0
:101CA400FA25DF3F31F4CF3F21F4A72FBB277F91E3
:101CB400E0CF7395703899F7F8CFB13011F0A77071
:101CC400A06CA0937C00A0917A00A064A0937A00F9
:101CD400A0917A00A6FDFCCFA0917800B091790084
:101CE4000895BB3020F4BA3028F0A83C18F0AFEFC8
:101CF400BFEF0895C8EDD1E0CA0FDB1FA881BB2751
:101D04000895B33018F4B23010F0A7FD15CEDF9368
:101D1400CF93CCE3DDE0CA0FDB1F0E94973FA62FD1
:101D2400BB270895B43021F4BB27AC91BB27089599
:101D3400B83050F0FF93EF93F091F010EEE0F7FF1E
:101D44000995EF91FF910895AF3F11F4A0B1EECF43
:101D5400A770A395B0B1B695AA95E9F7AA27AA1FCB
:101D6400E5CF7AB577700E943040BB27A52F80302D
:101D740009F08FE00895ED01DC3040F40E947040DA
:101D8400BB27A42F803009F082E20895E0E0F4E854
:101D9400EC0FFD1FA491BB2708957A2F0E944E409B
:101DA400803009F08FE00895AB2FBB270895CA2F28
:101DB400AA27BB27C03019F4A091220148C0C13022
:101DC40029F4A0912201A030E1F341C0C23039F4DA
:101DD400A0912201A030E1F7A091230138C0C330C3
:101DE40019F4A091200133C0C43039F4C09120010A
:101DF400C0FD1196C2FD11972AC0C53039F4C091B7
:101E04002001C1FD1196C3FD119721C0C63049F4CC
:101E1400C0912201C23E09F41197C33EC1F4119648
:101E240016C0C73049F4C0912201C43E09F411968A
:101E3400C53E69F411970BC0C83019F4A091210173
:101E440006C0D0912201CD17E1F7AC2FBB2708952E
:101E5400BB27A13021F4A0916D01A3950895A23070
:101E640021F4A0916E01A3950895A0916F010895A6
:101E74006F927F924F930E94BE404030A9F0342F5E
:101E84003395ED010E94B31C803071F521963E011B
:101E94001A2F0027A02F0E9428430E9407411417DD
:101EA40021F003950317B1F71CC0E3010E94B31C92
:101EB4008030D1F4A03091F02A2FA02F0E94BA4391
:101EC400E3012196E8E8F1E00E94B31C803061F45C
:101ED400B191AB1731F721962A95B1F7A02FBB2703
:101EE40002C0AFEFBFEF88274F917F906F900895A6
:101EF400AA0FAA0FBA2FAA27C0E0D6E0CB27CC0F8F
:101F0400AA1FCB2FBB0FDA95C9F7AA0FAA0FBB27BD
:101F14000895AA95A53048F40A2EA0E3BDE0A00DCB
:101F2400A00D0D901D90D0010895AA27BB270895F8
:101F3400C8E7D1E008811981AA81BB8182DDB7FBA2
:101F440068DD2D010C811D81AE81BF817ADD8201A6
:101F540091DD0C811D81A885B985F90172DD59DDFA
:101F64002D0156944794E40DF51D421D521D422C3B
:101F7400522C320100E2EE0FFF1F441F551F441C78
:101F8400551C661C771C4A165B066204720428F012
:101F94004A1A5B0A62087208E3950A9561F7DF0141
:101FA4000EF439CD088119814DCD0E9411028D01A5
:101FB4000C940C020F70003009F40895AA0FBB1F93
:101FC4000A95F9CF0F70003009F40895B695A795D6
:101FD4000A95F9CFFCE0E0EAA0E0B4EBA193BA954E
:101FE400E9F7F1E0E8E6B0E1A193BA95E9F7FDE09D
:101FF400ECE3B0E0A193A193A193BA95D9F7DD24C2
:10200400CC2420921B0120921901AEE0A093380148
:10201400ACE3A0935001AEE2A0935101AFEFA093C3
:102024007701A0931001209213010E944B34209257
:102034005C01AFEFA0935201A0935301A2E0A093DF
:102044003F01A6ECA0937A004091490140934601D8
:10205400409343010E94A5789C2D0E94AF7821D023
:10206400803039F4AC2DAF35B8F39CE020925C019C
:102074000895C0926D01D0926E0180936F018130FA
:1020840051F020925C01409177014F3520F4DD241A
:10209400C42E8827E1CF9CE020925C010895F701CB
:1020A4002EC0F1E0E0EB209236018827AD2DBB274E
:1020B400AB1729F171917F3FF1F07F3511F40C9446
:1020C400221C7C31D1F07E31C1F07D31A9F07F3109
:1020D40099F0773281F0723241F471917F3F59F077
:1020E400773249F07232C9F7E5CF7A3319F7B395ED
:1020F400AB1701F704C032C071917191DBCF7091BD
:10210400390170FD03C0803031F015C081E07E7F5D
:1021140070933901089572FF11C0AB7F7093390138
:10212400A0914A01A53011F0A03011F40E941F20A3
:10213400A0FF04C081E00F900F9008950E9485399C
:1021440070911301703039F0A0911001DA9420924B
:1021540013010C94FA1371917F3F19F4DD24C39495
:1021640008957F3511F40C94221C77FD2CC0703235
:1021740031F27A3311F4D394C2CF773209F4BBCF5E
:102184007134D8F07B3528F070527134B0F07B355F
:10219400A0F4672E0E9414197D3379F490DA80300C
:1021A40069F4762D7154770FDCE0C0EAC70FD21DB5
:1021B400A993B99375CFEF91FF9187E00895703893
:1021C40010F487E06CCF7F01EDEEF72FFF73EF0F74
:1021D400F0E1F21D09944AC0F3C06FC22FC10AC1D5
:1021E4009EC2CDC20EC7DAC2DEC2E5C236C060C628
:1021F40074C6F4C267C387C2F0C31DC475C164C486
:1022040077C47FC4D4C15FC287C495C49CC460C56D
:102214004BC1DCC04DC226C1FBC49FC425C0FEC453
:1022240016C512C28BC2C3C51DC011C66EC379C305
:102234006EC168C6C4C64AC717C61DC61CC224C51B
:1022440030C618C14FC289C3A1C296C4A0C43CC140
:102254006EC118C688C183E1089576FD0C94C91A2D
:102264000C9497190C948D180C94AE190E941E1995
:102274009CE0732C20923601B191B032E9F3BA3369
:1022840021F0B73211F0B03858F0319770FC0E9449
:102294009D3440913601453010F00E94FA3F00CF42
:1022A400BB3311F47724E8CFBC3291F4409136016A
:1022B400403031F40E94DE34BA2DB770D9F706C02D
:1022C4000E94DE34B0913701B770D1F77724D4CFB0
:1022D400732CB332B9F42092780120927901EFD9AA
:1022E4004A2F40933601453008F4C6CF0E94FE3F82
:1022F400683059F5509136015E7F0E940040683184
:1023040021F5BACFB03419F50E94DC18409136019A
:10231400433018F40E949736AFCF39F4A093780174
:10232400B0937901A0933701A7CF5FEF0E940040DB
:10233400683259F45A2F0E940040683231F45B2FFE
:102344000E940040683209F497CF8FE00895B132BB
:1023540029F4B5D99A2F90CF98CF8ECFB23241F4C9
:1023640041914F3FC9F34232C1F30E94DF34F8CFA9
:10237400B63291F4A4D9B33010F082E10895CCE3DD
:10238400DDE0CA0FDB1F4991403029F00E94DF34A1
:102394001196B330C0F370CFB53229F490D94A2FD7
:1023A4000E94DF3469CF31978AD9803009F00895CB
:1023B400903818F40E94DB335FCF0E9436345CCF30
:1023C40076FD0C94B11A0E944B3469CEA2E0B1E0C0
:1023D400B7D6B0917801BF70A13041F0A0917A01D5
:1023E400A295A07FAB2B0E94873359CEAB2F0E94BE
:1023F400AC3355CE76FD0C94791A0E940E1CA09332
:102404007201B0937301A0917A01B0917B01A09302
:102414007801B093790100917C0110917D0112152E
:10242400020549F00E94B51C0E94DB1C803029F48F
:1024340003191209F4CF33CE0ECF089576FD2FCEB3
:10244400A5E0B4E07DD60E9476197F93A2D6E093EE
:102454006B01F0936C010E9417387F9170933801DF
:102464001ECEF9CE76FDDCC10E94021CA170A093A1
:10247400190115CE76FD10C0A5E0B4E061D634D7BD
:102484007F9387D6E0936B01F0936C010E94303800
:102494007F917093380103CEA1E0B1E051D6A091B1
:1024A4007801A093FF10FBCDA5E0B4E049D61CD77A
:1024B4007F936FD6C0936B01D0936C010E942D3D26
:1024C4007F9170933801EBCDA5E0B4E039D60CD7F9
:1024D4007F935FD6C0936B01D0936C010E94623DE1
:1024E4007F9170933801DBCDA3E0B2E029D6FCD60E
:1024F4007F93B0917801A0917A01A0936B01B0937E
:102504006C010E94B3367F9170933801C8CDA5E069
:10251400B4E016D6E9D67F933CD6E0936B01F093F2
:102524006C010E9492387F9170933801B8CD76FD8A
:102534000C94EC1BA0914A01A03011F08CE1089599
:102544000E94021CCCE3DDE0CA0FDB1F409138017E
:102554004F93AF92BF920E94B03DBF90AF904F9106
:10256400409338019CCDA0914A01A03011F08CE138
:1025740008953CD657D67C32C1F47F010E94021CD8
:10258400CCE3DDE0CA0FDB1F409138014F93AF92DB
:10259400BF920E94F33DBF90AF9091D2499329928C
:1025A4004F914093380188277ACD87E078CDA09168
:1025B4004A01A03011F08CE1089518D637D67C3248
:1025C400A1F7A1E0B1E0BDD5AF92BF92409138012F
:1025D4004F937F930E947623403079F10E94D61E58
:1025E400A0913801A695AF700E9496250E947E3670
:1025F40003020000A0917801B0917901CCE3DDE001
:10260400CA0FDB1FA6E14991403230F0403820F474
:102614000E94DF34AA95B9F70E9433230E94F91E61
:102624004D3E59F04CD2799329927F914F9140932A
:102634003801BF90AF90882732CD41D27FEF799394
:102644007993F3CF87E02BCDA3E0B2E079D54CD6D4
:102654007F93D0916C01C0916B01F0917801E0916E
:102664007A01E0936B01F0936C010E9492387F91A0
:102674007093380114CD76FD0C94F51B0E94141C44
:1026840088D5E8940E94D0370ACD0E94141C81D5C5
:1026940068940E94D03703CD0E94141C7AD50E94FE
:1026A4004338FDCC0E94141C74D50E946F38F7CCBB
:1026B4000E94021C0E94B833F2CC0E94021CA1505A
:1026C400CA2EDD24089576FD06C00E94021CA15086
:1026D400A0937701E4CC0E94021CBA2F68940E9454
:1026E4008F3BDDCCA7E0B2E02BD5C8E7D1E0B881C1
:1026F400EA2FEA952296A8810E949C33B395EA9525
:10270400C9F7CDCCA8CD0E94021CA7700E94233328
:10271400A0914A01A73010F40E944B34C0CC76FD3E
:102724000C94371B0E94021CB03019F4A03009F439
:10273400B6CC0E94BA381197F7CF8DCD76FD0C94A4
:10274400FB1B20923F010E94141CCCE3DDE0FE0140
:10275400B33098F4CA0FDB1F00917A01A00FB21DA9
:10276400A00FB21DB33048F4EA0FFB1FA0917C0107
:10277400B0917E010E94D03F92CC82E190CC76FD54
:1027840097C620925C01BF91BF91089576FD0C9489
:102794002E1B54D5AB2B09F4AECC82CC76FD0C9415
:1027A400961A4AD57DCC76FD0C94EA1AF70102D527
:1027B4000E94973675CCA2E0B1E0C2D429F400900F
:1027C40053010092520105C0B0917A01E8940E942D
:1027D4008F3BA09178010E94C23862CCA6E0B1E0A0
:1027E400AFD4B1E0EAE7F1E05ED0A0917801AA9518
:1027F400AF3510F08AE053CCB0917001B93010F0CD
:102804008DE04DCCAF93DAD0B064B993BC2DB993BD
:10281400B0914901B993DD24CF9008950C94881B9D
:10282400A7E0B2E08DD47232C9F3B2E0ECE7F1E094
:102834003AD0409178014A950E9430794E3481F41F
:10284400F695E795A0917A0154FF06C0EA0FF21DB0
:1028540055FF02C089E208957096E89409951FCC4B
:10286400A0917A01AA95AF35B8F7B0917801BA95DD
:10287400B770B0934301B0917001B93010F08DE09E
:102884000ECCAF939BD0B064B993BC2DB993B091E7
:102894004601B993DD24CF90409143014093460112
:1028A4000E94A5780895C0E3DDE04A2F4B1B4093B6
:1028B4003A0D403009F40895519159935191599327
:1028C4004A95F7CFA1E0B0E03BD4B0917001B030AD
:1028D40011F48CE00895A13041F4A0917801A09303
:1028E4002E0DA0917901A0932F0DBA956FD0B093BE
:1028F4007001B991B6FFEDCFBF70DB2EC99049913D
:10290400409346010E94A5780895B0917001B930B2
:1029140010F08DE0C4CB52D0B062B993BC2DB99302
:10292400BECBB0917001BA95A0F050D0B991B5FF6B
:1029340010C084D4AB2BB091700121F4BA95B0933C
:102944007001AECBBA9542D0A991C990AF70DA2E7E
:1029540008958EE0089587E0089576FD0C94521C46
:102964006BD460D47134B8F37B35A8F77154770F06
:10297400672E58D47D3379F70E94610B803009F0BB
:102984000895DCE0C0EAC60DD21DA993B9934AD4D8
:10299400733C09F70E94610B2D01803009F0089502
:1029A400B0917001B93010F08DE0089507D0B0688F
:1029B400B993C99269924992599272CB07D0B3954F
:1029C400B0937001BD2DB395BF700895CCEFDCE0DA
:1029D400A5E0AB9FC00DD11D0895703C10F00C9480
:1029E40047132AD4B0917001B03011F48BE00895EC
:1029F400BA95ECDFB991B7FFF9CFBF700B2E5990A0
:102A04007991BCE0A0EAA70FB21D0D911D91030DB1
:102A1400121D1E930E93A991B99111960A1741F4B0
:102A24001B1731F4B0917001BA95B093700138CB93
:102A3400C52CD02C0895A0914A01A03011F08CE14E
:102A44000895FAD3BFEFB0938801B191B032E9F39E
:102A54004B2FBF3F21F40E949D34319721CBBA33D1
:102A6400D1F3BB3391F3BC3231F40E94DE34BA2D7E
:102A7400B770D9F7EACFB23241F441914F3F59F3DD
:102A8400423219F30E94DF34F8CFB134B0F0BB35D1
:102A9400A0F4B154BB0FB0936A01B081B13418F003
:102AA400BB3508F40AC0CDD3DCE0C0EA10916A015A
:102AB400C10FD21DA993B993C8CF87E00895C091DF
:102AC4007201D0917301089576FD0C944E13B6D320
:102AD400803009F0E5CA4A2F4B2BE1F340912E01D7
:102AE4004030E1F340912E014030E1F71197F3CFEC
:102AF40076FD0C945413A2D3A0932F01B09330010C
:102B0400EACF76FD0C94531B71D3A0912F01A993A6
:102B1400A0913001A993C4CA76FD0C94801C8ED375
:102B24004A2F0E94443A7FD37C3221F47BD30E9403
:102B3400610BF6CFB5CA76FD0C94651B0E94AF3AC3
:102B4400A42FBB273CC6F70143D34A2FD73010F03C
:102B5400C03D10F40E947940A3CAF70139D35A2F1B
:102B6400DE017AB577700E944340763020F40E94EB
:102B7400BA380E94BA3894CA76FD0C94C61B5ED348
:102B840079D616F086E208958827A1B989CA76FD18
:102B94000C94D71BF7011CD3D23019F40E94A01C4B
:102BA4007FCAD43019F4DD27A88379CAD83048F015
:102BB400F091F010F7FD2AC0EFE00995803031F371
:102BC40008950E943C1C06F7D030B1F4BC2FB770B6
:102BD400B39577276FE7A0FD70E8A0FD6FEF77FB53
:102BE400770F70F967FB660F60F9BA95C1F702B108
:102BF400072B062302B953CAD13041F4B2B1C095B0
:102C0400BC23C095CA23BC2BB2B949CA88E2089533
:102C140076FD06CE13D30E94263A42CAE7D2099122
:102C240019911058FFD27C3281F4D2D2B058D058C6
:102C3400C017D10708F08E01A017B10708F48D0161
:102C44003EDF1058099319932BCA86E00895A0918A
:102C54004A01A63029F0A370A03011F08CE1089548
:102C6400C5D23E01DFD27C3281F7A4D2C8EDD1E0D7
:102C74007EE17B9FC00DD11DCA0FD21DA881BB2749
:102C8400E301A993B9930CCAA0914A01A370A0309F
:102C940011F08CE10895AAD23E01C4D27C32A9F687
:102CA40089D2C8EDD1E07EE17B9FC00DD11DCA0F52
:102CB400D21DA2EBCA0FA2E0DA0FBB27A881A6950A
:102CC400BA2FA777B295B078AB2BD9CF86E0089509
:102CD4008DD23E01A7D27C32C9F76CD2C8EDD1E0C7
:102CE40070914A0177707030E9F4AF93BF93A69561
:102CF400B6957EE17B9FC00DD11DCA0FD21D788190
:102D0400BF91AF91A0FD7695B0FD7695B0FD769517
:102D1400A2EBB2E0CA0FDB1FA88170FFA295A695B3
:102D2400AF70ADCF7130B9F4AF93A695A695A695C3
:102D340075E17B9FC00DD11DCA0FD21D7881AF9163
:102D4400A2FD7295A1FD7695A1FD7695A0FD7695DF
:102D54007170A72FE5CF7230A1F4AF93A695A69515
:102D64007EE17B9FC00DD11DCA0FD21D7881AF912A
:102D7400A1FD7295A0FD7695A0FF76957370A72F9F
:102D8400CFCF733071F4AF93A6957AE27B9FC00DD9
:102D9400D11DCA0FD21D7881AF91A0FF7295A72FC4
:102DA400BFCFAF93A695A695A69570E1C2CFA0918B
:102DB4004A01A63029F0A370A03011F08CE10895E7
:102DC4002BD5B33010F082E10895B23039F4A73F27
:102DD40028F082E1089581E208953DCACCE3DDE064
:102DE400CA0FDB1FC0936601D0935501AC81A0309C
:102DF40091F3AE3180F7BB81B03069F3B73158F746
:102E0400C0917801D09179012596BA9F000C111CCC
:102E1400000C111CC00DC11DD330E8F6D0917A010D
:102E2400C0917C01C0935401D0935701CF3F51F01E
:102E3400DF3F41F0CA0FCA95CE3138F4DB0FDA9583
:102E4400D73118F40E944D3E2AC986E10895A09115
:102E54004A01A03011F08CE10895EED1A09139011E
:102E6400A460A09339011CC9D7D40E9415268030D0
:102E740009F415C90895D0D40E941E26803009F49F
:102E84000EC90895A3E0B2E05BD1A33021F0E3C9F9
:102E9400A4E1A0937C010E940326803009F4FFC8BA
:102EA4000895AED40E940C26803009F4F8C8089521
:102EB400ADD440917A01CCE3DDE0403041F0D395CC
:102EC400413029F0D395423011F082E108950E94F7
:102ED4003926803009F00895E2C898D440917A01E7
:102EE400CCE3DDE0403041F0D395413029F0D39577
:102EF400423011F082E108950E944426803061F34B
:102F0400089559C0F7010E940E1C90917801B09168
:102F14007A01A0917C01A09374010E94FE3F683065
:102F240081F790FF2BC0592F0E940040603449F76D
:102F3400A030D1F0DDE0CCE3409174014B0F4A1B8B
:102F4400C40FD21DA13039F00E940440603599F5B8
:102F54005883AA95EFCF0E940940683561F55883DC
:102F64000E94FA3F0C9452100E940440603519F5F7
:102F74005030B1F350937401A52FDCCF592F0E9428
:102F840000406831C1F43A2FDDE0CCE34091740194
:102F94004B0F4A1BC40FD21D5881503011F43030EE
:102FA40031F00E940040683231F4AA9569F70E941A
:102FB400FA3F0C9452108FE00E94FA3F08953ED1DC
:102FC400A0937801B09379012ED17C3249F43196E3
:102FD40029D1723239F031970E94610BEAD4F4CFCF
:102FE4000C9452107191723231F07F3F21F0BB2763
:102FF400A72FDFD4F7CF7081E7CFA43099F40C94D6
:10300400E219A7E0B4E09CD0B0917801B0935801E4
:10301400B13051F0B03031F0B23019F1B330F9F1D0
:10302400B73058F385E10895A730E1F7C8E7D1E058
:10303400BA81B0935501BC81B0936601BE81B0934F
:103044005601B885B0936701BA85B0935701BC8522
:10305400B09354010E94D13B803009F008950C9440
:103064005110A630F9F6C8E7D1E0BA81B093550102
:10307400BC81B0936601BE81B0935601B885B0930C
:103084006701BA85B0935401BB85B09357010E9480
:10309400D13B803009F008950C945110C3CFA43073
:1030A400E9F7C8E7D1E0BA81B0936601BB81B09378
:1030B4005501BC81B0935701BE81B09354010E9465
:1030C400D13B803009F008950C94511076FD0C9496
:1030D4002F1CA0914A01A03011F08CE10895F70152
:1030E40077D0C0937801D093790120917401A2170D
:1030F40008F42A2FA8E8B1E0203041F04D918D0169
:10310400A42FBB2756D4D8012A95F6CFAA27BB27CC
:1031140050D40C945210A0914A01A03031F0A43044
:1031240021F0A63011F08CE108956AD3A0917801C2
:103134004A2F43700E940F3F0C9451100C942D1190
:10314400F701DF93CF93BF93C8E7D1E040E05A2F54
:10315400DF93CF934F935F930E94610B5F914F91E5
:10316400CF91DF91A993B99343955A95503031F09B
:1031740071917032E9F37C3259F33197A42F7F01B6
:10318400BF91AB1718F4CF91DF9183E1CF91DF9119
:103194000895D0917801C0917A01F0917C01E09179
:1031A4007E01C0936601D0935501E0936701F093CB
:1031B40056010895A2E0B0E0C4DFA23029F4B09132
:1031C4007801A0917A010895AF91AF910C942D11DB
:1031D400A2E0B0E0B6DFA230B9F7C0917801D09197
:1031E4007901A0917A01B0917B010895F7011AD079
:1031F4007134A0F07B3560F47154770FDCE0C0EAE1
:10320400C70FD21DC0937201D09373017F0108953B
:10321400713620F07B3710F47156EFCF8F918F9178
:1032240087E0089571917032E9F30895F7017F0101
:1032340071917032E1F30895F7010895F7010C9448
:10324400610BEF93FF930E945039FE0100E00E944E
:10325400F53870913901713011F4872F09C04A3E55
:10326400E9F400937401003031F4AA27BB278827BE
:10327400FF91EF910895C8E8D1E0A191A9930A952F
:10328400E1F7AFEFA9930E941C1DE0EBF1E00E946F
:10329400610B8D010E94AF78D801E9CF4C3E49F40F
:1032A4000030A9F2AA940E945039A0E2A8830A959A
:1032B400CECF403260F24B3750F6AA2DAD3138F6FE
:1032C4000E94DF340395C3CF92E0BB27AC2DA395B6
:1032D4000E94DB334AE30E94DF34BB27AD2D0E94FA
:1032E400DB330E94DE34089570913801A0FF089505
:1032F400A33029F4A0917C010E94AC330895A53039
:1033040019F4A0918001F8CFA0918401F5CF0E9417
:103314002726403011F466270895409380010E94C7
:10332400CB25413009F066270895A2E0B1E008DF1B
:10333400B1E0A13011F0B0917A01A0917801A150CF
:10334400A0931001B09311010E94BA38B0931201F6
:10335400209213010C945110A3E0B2E0F1DEC0916D
:103364007801D091790140917A0108EC1AE028EDB6
:1033740031E0A23019F41CD00C94511060917C01FE
:10338400F0917B01F170E0917A014CE3E40F4DE0A0
:10339400F41F4427C40FD21D41910AD041914038F3
:1033A400C8F34058C40FD21D6A9551F70C945110BC
:1033B400C017D10720F4DE01A20FB31F4C93089568
:1033C400FF93EF930CE310E120EA3CE0B091780125
:1033D400B43019F5E8EDF1E0A0917A01B0917B01E8
:1033E400BF70AE0FBF1FC0917C01D0917D01DF7013
:1033F400CE0FDF1FE0917E01F0917F01A217B3078A
:1034040040F4C217D30728F4319718F00D900992AD
:10341400F5CFEF91FF910C945110B53009F5E8ED1B
:10342400F1E0A0917A01B0917B01BF70AE0FBF1F94
:10343400ECE3FDE0C0917C01D0917D01DF70CE0F03
:10344400DF1FE0917E01F0917F01A217B30708F717
:10345400C017D107F0F63197E0F20D900992F5CF3D
:10346400B63011F5ECE3FDE0A0917A01B0917B0157
:10347400BF70AE0FBF1FE8EDF1E0C0917C01D091A9
:103484007D01DF70CE0FDF1FE0917E01F0917F019F
:10349400A017B10740F4C217D30728F4319718F0E6
:1034A4000D900992F5CFB5CFEF91FF9185E1089585
:1034B400A3E0B2E045DE70914A0150917A01409157
:1034C400780160917C01763021F0743041F00C94E5
:1034D4005110A33051F40E94AA3B0C945110A23015
:1034E40021F40E94BE3B0C9451100C942D11A2E0C7
:1034F400B2E026DE0E94D425803009F008954031E0
:1035040021F0483111F083E2089590917A019A955F
:1035140070914601791731F0709178010E94A024CE
:103524000C94511085E20895A2E0B2E009DE0E94F5
:10353400D425803009F008954C3F11F087E10895B7
:10354400709049017091780190917A019A959093C5
:1035540049010E946B24709249010C945110A2E01D
:10356400B2E0EEDDA0E8B2E060917801C0917A01AA
:10357400D0917C01CA17DB0740F4ACE3BDE0CA0F6D
:10358400DB1F0E94BD3F0C94511082E10895A7E017
:10359400B6E0D6DDA9DE7F93E8E6F1E047D0C0933C
:1035A4006B01D0936C01E0917A01F09178010E9453
:1035B400923822D0C0916B01D0916C01E0917A01D4
:1035C400F09178010E9492387F9170933801C5CFB1
:1035D400A7E0B6E0B5DD88DE7F9304D07F917093D9
:1035E4003801BBCFE8E6F1E021D0DE01E8E6F1E006
:1035F400A383B4830E94B336E8E6F1E0A08DB18DD5
:10360400C28DD38D2196AC17BD0708F0089511968D
:10361400A08FB18F0BD0E0916B01F0916C01C0933E
:103624006B01D0936C010E949238E6CFA08DB18DCE
:1036340031D0048911270E942F0DD089DB1BA08D66
:10364400B18D9D979D970E944C1B068911270E945E
:103654002F0DC289CB0F0895D3D0A0FF0E94A03BA9
:10366400A0FD0E94A63B0C945110C0DDCF93DF93C4
:10367400D9DDA5E0B0E065DDA53041F40E949A0FE4
:10368400DF91CF91A993B9930C945110DF91CF910D
:103694000C942D11FF93EF930E945B0DEF91FF911A
:1036A4000895A4DDBFDD7C3259F4A1E0B1E049DD29
:1036B400A09178014BD003DA599329920C945110BC
:1036C40087E00C94511092DDADDD7C32C9F7A1E0A6
:1036D400B1E037DDE0917801F0917901E894F038B8
:1036E40018F0E095E3956894EAD9A881B981E1508E
:1036F40048F01EF0AA0FBB1FFACF0B2E000CB79593
:10370400A795F5CFA883B9830C9451104191423207
:10371400D9F4EF014191423211F04F3FD9F77F01C3
:10372400409178014A950E943079F695E7954E3498
:1037340059F4A0917A0154FF02C0EA0FF21D709669
:10374400689409950C9451100C942D11F0E951E0F2
:10375400EDE0649163FD05C0EFE064916A1709F43C
:103764000895F45F5395593099F750E008954F93B5
:103774004A954770E6E0E49F4F91E8E0F8E4E00DF5
:10378400F11DE50FF21D0994F29902C087E2089534
:1037940055DD4A2F0E94503A46DD7C3221F442DD49
:1037A4000E94610BF6CF0C9452109927F29903C032
:1037B40087E20C9451100E94C63AA42FBB27409173
:1037C40022014D3E11F4AFEFBFEF10DDA993B99381
:1037D4000C94521015D0F29902C087E208950E9409
:1037E400773A0C9452100CD0A170A0936B000C94F7
:1037F400521006D0A0FBABB5A7F9ABBD0C94521088
:10380400A1E0B0E09DDCA13090F416C0A2E0B0E0ED
:1038140097DCA23060F410C0A3E0B0E091DCA330E8
:1038240030F40AC0A4E0B0E08BDCA43028F0A0910E
:103834007801B09179010895AF91AF910C942D1155
:103844007F01F091F310F7FD06C0E0E109958030A7
:1038540019F40C94511088E008950E94021C4A2F18
:103864004F3F19F42C9A0C9451100E948F402C98BD
:103874000C945110EF93FF936894F091F410F7FDBA
:1038840004C0EDE0E491E6FFE894F091F010F7FD58
:1038940004C0EDE0E491E6FFE894FF91EF91089510
:1038A400A5DCC0DC7C3241F593DC8E019D0107D997
:1038B4002E016627A8010E94B91C6A2EA9010E9444
:1038C400B91CB62DA03288F0B03260F0AB1719F4F1
:1038D40028D06395EFCF061B1209261B3209030D6E
:1038E400121DE7CF0FEF1FEF02C0061B1209E20102
:1038F400099319930C94511087E0089577DC92DCB6
:103904007C32D1F77F010E94021C9D010027112700
:10391400D6D82E01A9010E94B91CA03240F301D0CF
:10392400F9CF030D121D12FD05C0230D321D32FD0A
:1039340001C008958F918F9182E10895AF3F29F4DA
:103944002CBCACE5ACBD2DBC08952CBC2DBCA6FD97
:103954003DBCAF73A064ACBD0895BDB5B7FFFDCF4A
:103964000895AE0104C04091720150917301CF9348
:10397400DF935330A1F03BD0533029F0A991BB27FA
:103984000EF4B9914CC0F091F410F7FD40C0E1E1A0
:103994000995AF9343950995BA2FAF9140C0F09123
:1039A400F410F7FD34C0E1E10995BB2738C0AE013E
:1039B40004C04091780150917901CF93DF93533043
:1039C40079F015D0533021F0A9930EF4B99324C0A3
:1039D400F091F410F7FD1BC0E2E10995AB2F05C08F
:1039E400F091F410F7FD13C0E2E1099515C05430CD
:1039F40030F4E894DDE0CCE3C40FD51F0895689457
:103A04005450440F551F5430A8F3AF91AF91DF9138
:103A1400CF91AFEF82E10895C8E7D1E002C0C2E7D9
:103A2400D1E008801980030C121C08821982DF91EE
:103A3400CF910895A0EBB1E04FEF52E24D935A9528
:103A4400E9F7A0EBB1E0C8E8D1E0C83A18F4A03D2A
:103A540008F401C0089548814032E9F04A33D9F0AE
:103A64008DD04F3FB9F34E3F81F374D04F3F91F364
:103A7400403059F7A1D0403041F740D0403029F7C9
:103A84000DD0403011F74991413618F04B3708F406
:103A940040524D93DACF21964D93D7CF488140338E
:103AA40020F04A3310F4405302C044270895642F91
:103AB400772721964881403380F04A3370F440538D
:103AC400660F771F0B01660F771F660F771F600D58
:103AD400711D640F721D2196EDCF703029F04DE1F8
:103AE4004D937D936D9308956A3020F04CE14D938E
:103AF4006D930895605D6D934CE10895488144325F
:103B040011F044270895662777272196588150336A
:103B1400B0F05A3310F4505308C05A3508F05052DC
:103B2400513468F0573458F457535F70529544E059
:103B3400550F661F771F4A95D9F72196E7CF703046
:103B440029F04FE14D937D936D9308954EE14D938C
:103B54006D9308954881423211F0442708952196C7
:103B64004D934991423219F44D9341E00895C73A77
:103B740018F042E24D9308954D93F3CF48814732B4
:103B840021F04F3561F04427089521964D93C83AAA
:103B940020F4A03D10F44991F9CF4FEF08954D93CF
:103BA40021964881413430F04B35C8F3413610F04A
:103BB4004B37A8F34EEF0895FF93EF93BF93AF9362
:103BC4005F93EEE0F2E50E014591403089F0689490
:103BD40057E0A591AE3239F0B991B13608F0B05240
:103BE400AB1709F0E8945A95A1F716F0E001EBCF72
:103BF4005F91AF91BF91EF91FF91403041F04D93B0
:103C04004F934881403211F42196FBCF4F91089590
:103C1400FF93EF93BF93AF935F930E0145914030B1
:103C240089F06894562FA591AE3239F0B991B13626
:103C340008F0B052AB1709F0E8945A95A1F716F0C2
:103C4400E001EBCF5F91AF91BF91EF91FF914030D5
:103C540049F04F9348814C3211F0403211F42196CF
:103C6400F9CF4F910895CBE8D1E0A0EBB1E040E269
:103C7400E2E24993EA95E9F7A297A03D28F44D9131
:103C8400423010F04F3F09F40895403220F040389C
:103C940010F486D0F2CF4C3121F4ED91FF2719D0E6
:103CA400ECCF4D3121F4FD91ED9113D0E6CF4E319F
:103CB40031F444E275D0ED91689449D0DECF4F31B0
:103CC40031F444E26DD0FD91ED9134D0D6CF50D093
:103CD400D4CFE8944FE24395E051F742E0F7E05F38
:103CE400F84D403311F05CD068944FE24395E85EA0
:103CF400F340E0F7E851FC4F16F0403311F050D098
:103D040068944FE24395E456F040E0F7EC59FF4FD6
:103D140016F0403311F044D068944FE24395EA50D2
:103D2400E8F7E65F16F0403309F03AD040E34E0F6F
:103D340037D00895E8944F2F42954F7011F012D068
:103D440068944F2F4F700EF011F00CD068944E2FE2
:103D540042954F700EF011F005D068944E2F4F70BD
:103D640001D00895405D4A3308F0495F19D00895A1
:103D7400EEE0F2E55591503009F40895451711F03D
:103D84003796F8CF5F9357E045914E3209F008D04B
:103D94005A95D1F75F915C3110F040E201D008955B
:103DA400CB3A08F4499308950E941102A0914A0164
:103DB400A0936E01AA270E942333A0913801A093F7
:103DC4006A01A0911B01A0936D01A0913601A093FB
:103DD400690120923601E8EDF1E0CCE3D7E0A4E6F6
:103DE400B5E0419149931197E1F70C940C020E94BC
:103DF4001102A0916E010E942333A0916D01A09342
:103E04001B01A0916A01A0933801A0916901A093BC
:103E14003601ECE3F7E0C8EDD1E0E1CFC6E1D4E050
:103E2400E8ECF6E041B150B168E0A9E4BFEA469598
:103E340010F4AFE4BFE2A993B193A0E3B0E85695C0
:103E440010F4A1E3BEE4AD8FB58F6A9571F70895C0
:103E5400452FA6E10E9487334F5B0E94DF344DE378
:103E64000E94DF34A7E10E948733C0EADCE0C50F7B
:103E7400D21DC50FD21DA991B9919DE00E94DB33DB
:103E84000895A3E10E949736A5E0C62FCA95AC9F7A
:103E9400CCEFDCE0C00DD11DA881A6FF08C00E94B4
:103EA4007E36FF5355422000A981AF7015C0A5FF8F
:103EB40006C00E947E36FF5250542000F5CF0E9467
:103EC4007E36FF464F5220004A8146954F5B0E9442
:103ED400DF340E94DE34A981BB27A39592E00E94BF
:103EE400DB334AE30E94DF34BB27A881AF700E9412
:103EF400DB33089520921B019927A7E00E948733A2
:103F04000E944B340E947E361200424954203031C4
:103F140032333435363700000E947E36130044496C
:103F240052000E947E3614004C455600E894ECE1A1
:103F3400F2E40E941F3BA5E00E9487330E947E3674
:103F440000004156522D43686970426173696332BF
:103F5400204D4F4E202020205000409143014F5CC3
:103F64000E94DF340E947E36FF3A000092E0BB27B5
:103F7400AC2DA3950E94DB330E947E36FF3A0000ED
:103F8400BB27AD2DA3950E94DB33EBE8F1E0C6EF30
:103F9400D1E0AEE141EFB191B03031F0BE8F4CAF22
:103FA4004993AA95C1F706C0B0E2BE8F4CAF4993BE
:103FB400AA95D1F7A7E10E948733C0E0D4E0E1E1FC
:103FC400F0E1E8940E94D0379DE050E0452F4C5F2B
:103FD400B42FAA270E9497363BDF53955D30B1F783
:103FE400452F4950B42FA9E00E94973631DF5395ED
:103FF4005A31B1F7A7E30E948733C3E1D4E0EDE17E
:10400400F0E1E8940E94D0370E947E3604135354A2
:1040140041434B3A00009927BB27A09170010E94AD
:10402400DB336CE0C0917001C61720F0C61BB4E00E
:10403400B60F27DF6A95B1F708950E941102AF9277
:10404400BF928F939F93B0DE0EDE54DF2CD088276F
:10405400A09139014D3E11F4A1601AC0443F09F406
:104064002BC070914A01703011F0753079F7413FDF
:1040740011F4AA270DC0423F11F4A46009C0433FC4
:1040840029F7B5DE0E94E638AA270E942333DDCF44
:10409400A09339010E94EE38AADE9F918F91BF90C0
:1040A400AF900C940C0220922301B8DE40912301BE
:1040B4004030D9F30C94853970E044240E94EE38E2
:1040C40037D0E894ECEFF1E40E941F3B0E947E3667
:1040D4001400506167653A00A091FF1090E00E94BF
:1040E40036340E94E638A09139014D3E11F4A160A6
:1040F400CFCF443F19F40E94EE38A7CF413F31F4AB
:10410400A091FF10AA95A093FF10DACF423F21F4AB
:10411400A091FF10A395F7CF463E11F47A95D0CF26
:10412400473E11F47395CCCF433F59F64394C6CF21
:10413400A7E00E9487330E944B340E947E36000021
:10414400417272617920566965772000A0E60E9469
:1041540087330E947E360200416472202000A0E56D
:104164000E9487330E947E360205202020202020D2
:104174002020204461746120202020202020202041
:104184002020000060E4679FE001D370FE0163E03B
:10419400A0E0B62F0E949736A6E00E948733DF0185
:1041A40091E00E943634A5E0B62F0E949736A5E030
:1041B4000E94873390E058E05F936F930E94B31C92
:1041C4006F915F9121964A2F0E94363440FE09C0B8
:1041D400A7E10E9487330E94DF34A5E00E94873361
:1041E40002C00E94DE345A9539F73896F370D370C2
:1041F4006395633169F608952045786974205061A8
:1042040067652D20506167652B202043686172200B
:10421400204D6F6E202002002045786974202020F4
:10422400476F2020205374657020205669657720DD
:1042340020417272617902002092360120924A0173
:10424400A5E00E948733C0E0D0E0EDE1F6E10E94F2
:104254006F38A0E50E9487330E947E3601024446EF
:104264004C4153482073697A653A20000E942726FE
:104274004F3749F40E947E36FF353132204B694274
:104284007974650011C04F3F41F40E947E36FF31BE
:10429400204D69427974650007C00E947E36FF3064
:1042A40020427974650012C00E94CB254130C1F0D0
:1042B400E4EDF4E40E94D43A413009F432C04530CC
:1042C40009F4BACF4230A1F731D0B6CFE4EFF4E429
:1042D4000E94D43A413009F424C04530B9F7ACCF38
:1042E400E6E9F4E40E94D43A413009F41AC04730B4
:1042F40019F40E948A22A0CF4A3011F417D09CCF1F
:10430400423011F46DD098CF433019F40E94D52275
:1043140093CF443019F40E941B238ECF453001F70C
:104324008BCFA0912201A030E1F708950E94EE3DC9
:104334004F466F726D6174204D656469756D3F0001
:10434400413009F00895A6E20E948733C2E0D8E024
:10435400EBE1FCE00E9443380E947E360903466F7D
:10436400726D617474696E672E2E2E2020202020B9
:1043740020000E947E360B0300000E94302680300D
:1043840001F50E947E360903466F726D617474698B
:104394006E672E2E2E20446F6E652100A2E70E94C8
:1043A40087330E947E360B0320202050726573737E
:1043B40020616E79206B6579212020000E94E63807
:1043C40008950E947E360903466F726D61747469A4
:1043D4006E672E2E2E204572726F72210000DECF82
:1043E400A0E60E948733C4E0D8E0E9E1FDE00E9442
:1043F40043380E947E360905417661696C61626CBE
:10440400653A00000E947E360A0546696C65733A77
:1044140020009CE00E94E825DF93CF93DF010E94F7
:10442400DB330E947E36FF202F000E942726A42F14
:10443400B0E011960E94DB330E947E360B05426C7D
:104444006F636B733A00AF91BF910E94DB330E949C
:104454007E36FF202F000E94F125A0EFA49FD001FB
:104464001197B03009F413970E94DB33A6E00E9441
:1044740087330E947E360C052020205072657373AA
:1044840020616E79206B6579212020000E94E63836
:10449400089520457869742020496E666F20426132
:1044A400636B7570526573746F7252657363616E7A
:1044B400010020202020202044656C6574652020A4
:1044C40020202020202020202020466F726D61743F
:1044D400204578697420466F726D61742020202015
:1044E400202020202020202052657363616E00006C
:1044F400204578697420202020202020202020209E
:10450400202020202020202052657363616E00004B
:104514007727EAD04030C1F006D30E947E360302EA
:1045240044656C6574652066696C65009AD04D3E7F
:1045340059F07093780136D34C3FC1F330D14130F8
:1045440019F4A72F97D266D308957727CDD040309A
:1045540049F1E9D2A0E1A0937C010E947E360302D6
:104564005361766520500000CAD27BD04D3ED1F015
:104574007093780117D3403E30F4403171F04831E4
:1045840061F0DDD0E3CF22D3D03021F4CC3010F46D
:1045940010D1DCCF6FD29DD10895F5D04130B1F662
:1045A40069D2A3D1089577279FD04030D9F3BBD2E5
:1045B400A2E1A0937C010E947E3603024261636BF8
:1045C400757000004ED04D3E69F370937801EAD2C5
:1045D400403920F4423161F0B2D0E6CFF7D2D03086
:1045E40021F4C03610F4E5D0DFCF44D207D20895C9
:1045F400CAD04130C9F63ED20DD20895772774D07F
:104604004030B1F090D20E947E3603024C6F616458
:104614002050000074D225D04D3E51F070937801A3
:10462400C1D2403121F0483111F097D0E8CF84D184
:104634000895772759D04030D9F375D20E947E3639
:104644000302526573746F7265000BD04D3E81F3A3
:1046540070937801A7D2423111F08AD0EBCFF2D116
:1046640008957727B1D007D10E94E6384D3E11F462
:104674002BD108954A3E09F40895403E19F40DD112
:104684007727F0CF413E21F408D170918001EACF21
:10469400443E49F4703041F300D17150472F4F70BC
:1046A4004F3001F3E0CF453E59F440918001471764
:1046B40009F4DACFF2D07395472F4F7099F2D3CF24
:1046C400463E29F4703180F2E8D07051CBCF473E9A
:1046D40051F4409180014F3031F04051471718F0A8
:1046E400DCD0705FBFCFC0CF0E942726403009F4D2
:1046F4001AC0409380010E94BA380E94BA3849D245
:10470400413009F001C008950E94AB3D2F44464C4E
:10471400415348206E6F7420666F726D61747465C6
:104724006400442708950E94AB3D2F44464C4153F6
:1047340048206572726F72210000442708950E9418
:10474400AB3D2F43616E206E6F74207361766520DC
:104754006F6E20746869730008950E94AB3D2F4EFC
:104764006F2042415349432066696C6500000895F7
:104774000E94AB3D2F4E6F204241434B5550206663
:10478400696C650008950E94EE3D604F766572770E
:10479400726974652066696C653F000008950E9423
:1047A400EE3D2F44656C6574652066696C653F0059
:1047B40008950E94AB3D2F4E6F2073706163652096
:1047C4006C656674000008955F936F937F93A72FC1
:1047D400A07FA0936C01A0916C01AF70AB5FBA2F66
:1047E400A4E00E949736A6E00E948733A0916C0152
:1047F400BB2795E00E94DB330E94DE34A5E00E94D3
:104804008733A0916C01A0937801CCD1B5D04F3FF0
:1048140061F1A0916C01A093780140E040937A018A
:1048240042E040937C018827FED1803091F4CCE3B0
:10483400DFE00E94DE345CE05F934991403808F089
:104844004EE2403208F440E20E94DF345F915A9510
:1048540099F7A0916C01A395A0936C01AF7009F036
:10486400BACF7F916F915F9108955DE00E94DE342D
:104874005A95E1F7EECF4F935F93C4E2D5E0472F0B
:104884004F705EE1459FC00DD11D52EF47E1599332
:104894004A95E9F75F914F9108954F935F93C4E26E
:1048A400D5E0472F4F705EE1459FC00DD11D5CE000
:1048B40044E059934A95E9F75AE043E159934A95FC
:1048C400E9F75F914F910895A0912201A030E1F79B
:1048D4000895709378014CE040937A0140E140934D
:1048E4007C018FD1803009F01ECF709378019091B4
:1048F4004901ECE0F0E99770929540EC949FE00D4B
:10490400F11D04913C9740E10E3409F448E155D17E
:1049140040E04F9300E0CCE3DFE0159119930A9552
:10492400E1F740937A0142E040937C0185D14F91B5
:1049340043954C3071F70895909149019770E0E0E8
:10494400F0E9929540EC949FE00DF11D40E04F9307
:1049540040937A0142E040937C017093780163D1E3
:10496400CCE3DFE00E94F07832964F9143954C30CF
:1049740071F778940C94FA790E9401024F93742F82
:10498400E2ECF9E44591403051F464E04DE20E94D8
:10499400DF346A95D9F74F914FEF0C94FA0147171A
:1049A40011F03396EFCF63E045910E94DF346A95AE
:1049B400D9F74AE30E94DF344F910C94FA01104274
:1049C4004153124255501455535216434838184116
:1049D40056521A47504C1C53414D1E4C424C2042D7
:1049E4004133224156332453583326564D332842FB
:1049F400553330545647325A58500000709378015A
:104A040040E640937A0142E140937C01FAD0803041
:104A140009F089CE709378014427E0E0F0E94F93E0
:104A2400CCE3DFE00024159019920A94E1F7409357
:104A34007A0142E040937C01FFD04F914395403688
:104A440071F7089540E0E0E0F0E94F9340937A0174
:104A540042E040937C0170937801E5D0CCE3DFE041
:104A64000E94F07832964F914395403671F77894CE
:104A74000C94FA790E9401024F93409138014093BB
:104A840081014CE440933801C6E0DAE0E7E1FCE060
:104A94000E9443380E947E360B0757726974696E10
:104AA4006720646174612E2E2E0040918101409331
:104AB40038014F910C94FA010E9401024F934091E6
:104AC4003801409381014CE440933801C5E0DAE0B9
:104AD400E8E1FCE00E9443380E947E360B06446104
:104AE4007461207472616E736665722E2E2E0000DE
:104AF40040918101409338014F910C94FA01CCE329
:104B0400CCE340914901942F4F5C0E94DF3440E292
:104B14000E94DF344BB54F9340684BBD0E9423790C
:104B24004F914BBD0895A4E00E948733C1E0D2E0C9
:104B3400ECE1F5E10E946F38A2950E948733089555
:104B440033D904D054D9089501D00895ECDFA2E0FC
:104B5400B3E00E9497360F901F90FF91EF91EE0FF4
:104B6400FF1F4591403019F00E94DF34FACF31978E
:104B7400F695E7953196EF93FF931F920F9271DDAF
:104B84004D3E19F0709378010DD008950090F51002
:104B94000895FCDF07FC03C0EF93E1E17EC00E94AF
:104BA40045420895F3DF07FC03C0EF93E2E175C0CB
:104BB4000E9426430E9407410895E8DF07FC03C0D2
:104BC400EF93E3E16AC00E9403410895DFDF07FC2D
:104BD40003C0EF93E4E161C00E9463420895D6DF0D
:104BE40007FC03C0EF93E5E158C00E94B04008956C
:104BF400CDDF07FC03C0EF93E6E14FC00E943541CF
:104C04000895C4DF07FC03C0EF93E7E146C00E94A8
:104C1400CB420895BBDF07FC03C0EF93E8E13DC03E
:104C24000E942E430895B2DF07FC03C0EF93E9E12D
:104C340034C00E9498430895A9DF07FC03C0EF9392
:104C4400EAE12BC00E9444430895A0DF07FC03C09F
:104C5400EF93EBE122C00E94BE40089597DF07FC6A
:104C640003C0EF93ECE119C00E94E24108958EDF86
:104C740007FC03C0EF93EDE110C00E94D3400E94F3
:104C8400C341089583DF07FC03C0EF93EEE105C041
:104C94000E948D410E94EF400895FF93F02D0995E5
:104CA400FF91EF910895A1E00E94263A20923601E7
:104CB40020924A01A7E00E948733C0E0D0E0EDE1F2
:104CC400F6E10E946F38A0E70E9487330E947E3687
:104CD40001024368697042617369633220636F6ED5
:104CE400666967706167650000270E9476782EB355
:104CF4003AB560916B0022FF216051D0E6E7FFE4F2
:104D04000E94D43A413009F40895433041F40E949A
:104D140085780E94BA380E94BA380C940000443E48
:104D240021F4013058F30A95E8CF453E21F40730C9
:104D340028F70395E2CF423009F7003031F46325B8
:104D440060FF232522FF2160D8CF013019F470E1E0
:104D54002727D3CF023019F478E02727CECF0730A6
:104D640031F4732F3F78705F7077372BC6CF0330E1
:104D740031F4732F73957770387F372BBECF04309F
:104D840021F4205C08F02064B8CF053019F472E0F7
:104D94002727B3CF063011F470E22727AECFA6E061
:104DA4000E9487330E947E36030153657269616CE9
:104DB4002073706565643A000E947E3605014932AD
:104DC400432073706565643A00000E947E360701D3
:104DD4005350492073706565643A00000E947E3622
:104DE4000901454550524F4D2061646472657373E7
:104DF4003A000E947E360B014C696E6520656E6434
:104E04003A000E947E360D0153657269616C204937
:104E14006E2F4F75743A00000E947E360F01536561
:104E24007269616C20496E7075743A000E947E3616
:104E340011014175746F73746172743A0000112723
:104E440090D0A2E1B3E00E949736E6E9FFE420FDAA
:104E5400749660FD3A960E94763683D024FD08C08D
:104E64000E947E360512313030206B487A0007C02C
:104E74000E947E360512343030206B487A0071D09F
:104E840023FD08C00E947E36071235204D487A2043
:104E9400200007C00E947E360712313536206B4849
:104EA4007A005FD00E947E3609120000432F4770BB
:104EB400405D0E94DF3455D0722F707C703839F415
:104EC4000E947E360B124C46202020000FC0703406
:104ED40039F40E947E360B1243522020200006C073
:104EE4000E947E360B1243522B4C46003AD021FDD1
:104EF40009C00E947E360D1273696D706C652020A6
:104F0400000008C00E947E360D127374616E6461E5
:104F14007264000026D025FF06C00E947E360F1260
:104F24005044330005C00E947E360F1250443100B5
:104F340018D00E947E361112505247200000432F91
:104F44004295477039F0405D0E94DF34A7E00E942B
:104F5400873308950E947E3611126F666620200002
:104F6400F5CFA5E0011709F4A0E50E948733139556
:104F740008952045786974204368616E67652053FD
:104F84006176652020202020202020202020202041
:104F940002003936303020283229000033386B348F
:104FA40020283229000031323030202831290000F5
:104FB40032343030202831290000AEE2A093380189
:104FC400C1E0D4E0ECE1F2E10E9443380E947E3675
:104FD400050500000E943C030E947E360603202043
:104FE40020202028632920323030362D32303135CC
:104FF40020202020202000000E947E36070320204D
:1050040020206279204A6F65726720576F6C667240
:10501400616D202020200000A2EAA09338010E94A4
:105024007E360903202020202020446564696361C2
:1050340074656420746F20202020202000000E94CA
:105044007E360A03466C6F7269616E2C2045726964
:105054006B20616E64204469616E612E0000AEE2D3
:10506400A09338010E947E360C0254686973207341
:105074006F667477617265206973206C6963656E0D
:10508400736564000E947E360D04756E646572203B
:10509400746865207465726D73206F66207468652A
:1050A40020000E947E360E04474E55205055424C37
:1050B4004943204C4943454E534520562E33200046
:1050C4000E947E360F035573652069742061742035
:1050D400796F7572206F776E207269736B2100008F
:1050E400A2ECA09338010E947E361107205052454D
:1050F400535320414E59204B455920000E94E63815
:1051040008959091490161E00E94AD3A50912201C5
:105114005D3E09F408954531B1F7E0E0F0E9977098
:10512400929540EC949FE00DF11DCCE3DDE050E05E
:10513400459149935A95E1F7CCE3DDE00E94BD3FE8
:105144000E94AD3A509122015D3E21F34630A1F711
:105154006395CCEBDDE00E94BD3F0E94AD3A5091D7
:1051640022015D3EB9F24630A1F763956931E9F653
:1051740044E00E94423A0E94AD3A08959091490158
:105184009770E0E0F0E9929540EC949FE00DF11DFA
:1051940045E10E94423A60E06F93CCE3DFE00E9475
:1051A400973F803041F0813061F1843251F145E123
:1051B4000E94423AF2CF46E00E94423ACCEBDFE052
:1051C4000E94973F803041F08130D9F08432C9F099
:1051D40045E10E94423AF2CF0E94F07878943296E8
:1051E40046E00E94423A6F9163956C30A9F60E94A2
:1051F4005B3A4430E1F746E00E94423A0E94BA38F2
:1052040008956F910E94BA38089502414253282E9E
:105214002E2E0353474E282E2E2E04535152282E41
:105224002E2E054E4F54282E2E2E06524E44282E36
:105234002E2E07414443282E2E2E08494E282E2E6A
:105244002E2E09585045454B282E0A54454D5028BA
:105254002E2E0B4C4F282E2E2E2E0C4849282E2E47
:105264002E2E0D4B4559282E2E2E0E455045454BBE
:10527400282E0F455252282E2E2E104152282E2E03
:105284002E2E1153494E282E2E2E12434F53282EC4
:105294002E2E134654595045282E144653495A4528
:1052A400282E155053544154282E16535049282E55
:1052B4002E2E174D454E55282E2E18565045454B2B
:1052C400282E1958524543282E2E1A4646494E4434
:1052D400282E1B44424954282E2E805052494E54A5
:1052E4002E2E81434C532E2E2E2E82474F544F2E5A
:1052F4002E2E83424F582E2E2E2E8441434F50592A
:105304002E2E8553594E432E2E2E86454E442E2E38
:105314002E2E8742434F50592E2E885448454E2EE8
:105324002E2E89504F532E2E2E2E8A4E4F54452EFC
:105334002E2E8B4F4E53594E432E8C525245414480
:105344002E2E8D5257524954452E8E474F53554257
:105354002E2E8F52455455524E2E90564D4F444545
:105364002E2E914E4558542E2E2E92494E50555461
:105374002E2E93504C4F542E2E2E94574149542E7A
:105384002E2E95545345542E2E2E96544745542E66
:105394002E2E974653454C454354984F4E455252F2
:1053A4002E2E99535055542E2E2E9A534745542E33
:1053B4002E2E9B45504F4B452E2E9C47455450490D
:1053C400582E9D434952434C452E9E434F4C4F52B9
:1053D4002E2E9F424F524445522EA0464F4E542EDD
:1053E4002E2EA150554D502E2E2EA258504F4B45C7
:1053F4002E2EA356504F4B452E2EA44C494D4954A6
:105404002E2EA547455443484152A6445241575471
:105414004F2EA7504C41592E2E2EA853505249546A
:10542400452EA95343524F4C4C2EAA425245414B50
:105434002E2EAB5245504541542EAC554E54494C3A
:105444002E2EAD445241572E2E2EAE49434F4D4D74
:105454002E2EAF444154412E2E2EB0435445585461
:105464002E2EB146524541442E2EB246575249542F
:10547400452EB343424F582E2E2EB4474554415423
:105484005452B54644454C455445B646424F582EB1
:105494002E2EB750414C45545445B8464F522E2EEB
:1054A4002E2EB949462E2E2E2E2EBA4449522E2E79
:1054B4002E2EBB4F55542E2E2E2EBC4643495243FE
:1054C4004C45BD414C4552542E2EBE464352454197
:1054D4005445BF41534B2E2E2E2ECE474F532E2EC6
:1054E4002E2EC03F2E2E2E2E2E2EC15853454E4406
:1054F4002E2EC2474F2E2E2E2E2EC3544F2E2E2E1E
:105504002E2EC44C4F4144502E2EC55343414C457E
:105514002E2EC643434841522E2EC742432E2E2ED2
:105524002E2EC853415645502E2EC94152432E2E7D
:105534002E2ECA4E4F2E2E2E2E2ECB5049452E2EB9
:105544002E2ECC5252442E2E2E2ECD5257522E2E6B
:105554002E2ECF5245542E2E2E2ED0564D2E2E2E7C
:105564002E2ED149424F582E2E2ED2494E502E2E39
:105574002E2ED3504C2E2E2E2E2ED44652414D4537
:105584002E2ED5484652414D452ED64C46494E44C2
:105594002E2ED74653454C2E2E2ED8564F4C2E2EFB
:1055A4002E2ED9544C454E2E2E2EDA4153484946C0
:1055B400542EDB45502E2E2E2E2EDC4750582E2EE8
:1055C4002E2EDD43492E2E2E2E2EDE434F4C2E2E14
:1055D4002E2EDF424F2E2E2E2E2EE043414C4C2EEB
:1055E4002E2EE143412E2E2E2E2EE258502E2E2EFC
:1055F4002E2EE356502E2E2E2E2EE44C494D2E2EBA
:105604002E2EE54743482E2E2E2EE644544F2E2EA2
:105614002E2EE7575241502E2E2EE85350522E2E46
:105624002E2EEB5245502E2E2E2EEC554E542E2E51
:105634002E2EED44522E2E2E2E2EEE49432E2E2E9D
:105644002E2EEF44412E2E2E2E2EF053504953452C
:105654004C2EF14652442E2E2E2EF24657522E2E0A
:105664002E2EF3424155442E2E2EF44741542E2E15
:105674002E2EF54644454C2E2E2EF6504147452EEF
:105684002E2EF750414C2E2E2E2EF85446494E44C1
:105694002E2EF95649442E2E2E2EFA45535055548B
:1056A4002E2EFB45534745542E2EFC4643492E2EA1
:1056B4002E2EFD45424155442E2EFE4643522E2E9B
:1056C4002E2E002E2E2E2E2E2E2E28B818954F93C9
:1056D4005F936F93FF93EF93DF93CF93BF93AF9356
:1056E4000F921F92FFB7FF93B0913D01B7FF5C98F3
:1056F400B7FD5C9AD9B1D3FBF59BD1FBB0F9F19B13
:10570400B325B0933D01C4E1D1E05F89A889E9895B
:105714000A881B88A00DE11DA88BE98BFFA1449189
:10572400AC89AF73AF3309F4452F5AA5BEADB59F0D
:10573400512D4503B0E8B10DB093B300E0912A01B7
:10574400F0912B0140912C0150912D01A52FAA0F0E
:10575400EE1FFF1F441F551F40F4ADE5EA27A5EDDA
:10576400FA27AAE24A27A5ED5A27E0932A01F093E3
:105774002B0140932C0150932D01830C921CEBA917
:10578400FF81EF23E8B97894EBB5F8A5F21529F079
:1057940090FC0CC08F1650F4BEC0F091F010E7E1FD
:1057A4000995FEF4C4E1D1E0EBB5F2EF8F1671F484
:1057B400409110014F3F51F0409112014A9521F45C
:1057C400409111013092130140931201FFE0E2FF76
:1057D400F2EF8F1639F45E98E3FFC8C0B2E8B093D5
:1057E4008000C4C0F3E1E2FFF5EF8F1639F45E9A4E
:1057F400E3FFBCC0B2ECB0938000B8C0FBE1E2FFB1
:10580400FFEF8F1621F4EFEFE0934701AFC0F2E012
:10581400E2FFF1EF8F1641F420924701F091F1106D
:10582400E1E2F7FF0995A2C0F9E3E2FFF7E08F1682
:1058340009F09CC0A8EDA883A1E0A9832E82882446
:105844009924AAE0A9AFA5E0E2FFA39542E3E2FF11
:105854004CE3BA8DB395BA1731F4BB27EB8DFC8DAD
:105864003196EB8FFC8FBA8FE885E395E41709F442
:10587400EE27E887F091F210E2E2F7FD02C0099505
:105884000EC0FDE8E0E0A0912801A7FDB096AD8927
:10589400EA0FF21DB491B21511F0A395AD8BBAA71E
:1058A40060913F016030B1F1B0915D01BA95B09360
:1058B4005D0181F5B0915C01B0935D01B09164012B
:1058C400BA95B093640131F5E0915E01F0915F0106
:1058D400C0916201D09163012197A191B1914B2FA5
:1058E400B295BF7019F0E8940E948F3B4F704093BB
:1058F40064010E94C238EC17FD0740F067FF6A9507
:1059040060933F01E0916001F0916101E0935E01D9
:10591400F0935F012BC0A0918400A83EE0F3A93E60
:1059240000F0AA3E00F0AB3E00F0AC3E00F0E5FD16
:105934001DC0E0914A01E3FD0C949B2EEE0FF6EAA4
:10594400EF0FFCE2F21D09940C943A2D0C94842D73
:105954000C94D42D0C940B2E0C944E320C943F2E9C
:105964000C94FF31F091F010E7E10995E091F71004
:10597400E7FF79C0A0912001A5FD23C0E091C000FC
:10598400E7FF67C0E091C600E0937101F5EFB491C1
:10599400B0FF32C0A7FF03C02092220157C0E338F2
:1059A40009F4E0E1F8E8EF77A4FFA6FDF395A4FF7E
:1059B400A0FDE068A1FDE068E491E0932101A0620C
:1059C40046C0E0912101E0932201E0932301EE3EE1
:1059D40019F4A2FD0C94B60140913901E33611F497
:1059E400A2FD4160E03711F4A3FD4260EC3F09F4ED
:1059F4004460409339012AC0E03F11F4A06827C0F5
:105A0400E03E11F4A06423C0E23131F4A6FD1EC0CF
:105A1400A160A7FDAE7F1AC0E93521F4A260A7FDFD
:105A2400AD7F14C0E43151F4A6FD04C0A460A7FD09
:105A3400AB7F0CC0A860A7FDA77F08C0E13121F4AB
:105A4400A061A7FDAF7E02C020922201AF71A09396
:105A5400200140916B0040FD0E94107840FF0E949D
:105A640045780C940278E0E20995F3CF0C94B82CB5
:105A7400A82DA530D8F3A0911401B0911501ED0122
:105A8400E2EBF2E0CE0FDF1FF6EFE0911A01FE0F1A
:105A94007F934F92EEE14E2E6991ED915491762FC2
:105AA4007295762757FD672768B9ED91000056FD7A
:105AB40076B9049055FD76B96991162E54FD76B9E0
:105AC4001294162653FD76B907FC61254A9452FDBB
:105AD40076B9502D712D41F760911B0168B94F9033
:105AE4007F91EE91F0911A01F395FA3029F4FF2792
:105AF400A0931401B0931501F0931A010C94B82CDF
:105B04000C94B82CA82DA530D8F3A0911401B09111
:105B14001501F82DF550CCE5DBE0F295FF70E5E1D9
:105B2400EF9FC00DD11D10901B01FD916991462F6F
:105B3400F0FD429548B9562F452FF1FD429548B9DD
:105B44000000452FF2FD429548B96991452FF3FDB8
:105B5400429548B90000452FF4FD429548B90D908F
:105B6400452FF5FD429548B90000452FF6FD4295B5
:105B740048B9F7FD5295462F00FC429558B9F02DCF
:105B8400EA95C1F618B8EE91F0911A01F395F23046
:105B940029F4FF27A0931401B0931501F0931A017F
:105BA4000C94B82CA82DA730D8F3A0911401B0916F
:105BB4001501D1E0FEE110901B01ED91CE2FC370D1
:105BC400588158B9CE2FC695C695C3705881E295B1
:105BD40058B9CE2FC3705881CE2FC69558B9C695E3
:105BE400C3705881ED91CE2F58B9C3705881FA957E
:105BF40041F718B8EE91F0911A01F395F33029F4B6
:105C0400FF27A0931401B0931501F0931A010C948B
:105C1400B82CA82DA53020F2A0911401B091150143
:105C24000F9310901B01EAE2D1E0CD9100000C2FFC
:105C34000295CF70F881F8B9C02FCF70F8810000B9
:105C4400000000000000F8B9CD9100000C2F02956F
:105C5400CF70F881EA9579F718B811970F91F09100
:105C64001A01F395F43029F4FF27A0931401B0939B
:105C74001501F0931A010C94B82CA82DA833D8F36D
:105C8400A0911401B0911501D0910001C0910101BE
:105C9400C295DC0FDE7EE0E110901B01FD914D2FDB
:105CA400F0FD429548B90000000000004D2FF1FDC1
:105CB400429548B90000000000004D2FF2FD4295C6
:105CC40048B9000000004D2FF3FD4295000048B98B
:105CD400000000006D2F4D2FF4FD429548B90000DF
:105CE400CD91F5FD62955D2F68B900000000F6FDC9
:105CF40052956D2F4D2F58B9F7FD6295C0FD429511
:105D04000000000068B9FC2F00000000EA9551F67D
:105D1400000018B8EE91F0911A01F395F23029F4CD
:105D2400FF27A0931401B0931501F0931A010C946A
:105D3400B82CD82DD730F0F0A0911401B0911501F2
:105D4400C0914D01F6EFE0911A01FE0FE395E09347
:105D54001A01EA3088F1EC3069F59396A0931401A6
:105D6400B093150120921A01D43130F4D0914C0132
:105D7400D0934D010C94B82CDF3188F4A1E4B2E047
:105D8400C0913A01D3E2CD9FA00DB11DCEE0A09306
:105D94001401B0931501C0934D010C94B82CDD3D52
:105DA40048F0CBE4AEE1B2E0A0931401B093150146
:105DB400C0934D010C94B82C0F931F932F93DD3D8A
:105DC40028F4DC2F0C2F1C2F2C2F05C028E61CE2F6
:105DD40008E8DCECCAE46C2F7C2F7295ED91E7FDAA
:105DE4006727EF775491ED9168B9172E56FD16B8D1
:105DF4006C2F7C2F729555FD16B8E7FD672754FD6F
:105E040016B8EF77000053FD16B8049052FD16B88B
:105E1400502DED9168B9172E56FD16B86C2F7C2FB6
:105E2400729555FD16B8E7FD672754FD16B8EF7750
:105E3400000053FD16B8049052FD16B8502DED9194
:105E440068B9172E56FD16B86C2F7C2F729555FD28
:105E540016B8E7FD672754FD16B8EF77000053FD29
:105E640016B8049052FD16B8502DED9168B9172E4E
:105E740056FD16B86C2F7C2F729555FD16B8E7FDAC
:105E8400672754FD16B8EF77000053FD16B8049049
:105E940052FD16B8502DED9168B9172E56FD16B85F
:105EA4006C2F7C2F729555FD16B8E7FD672754FDBE
:105EB40016B8EF77000053FD16B8049052FD16B8DB
:105EC400502DED9168B9172E56FD16B86C2F7C2F06
:105ED400729555FD16B8E7FD672754FD16B8EF77A0
:105EE400000053FD16B8049052FD16B8502DED91E4
:105EF40068B9172E56FD16B86D2F7D2F729555FD76
:105F040016B8E7FD672754FD16B8EF77000053FD78
:105F140016B8049052FD16B8502DED9168B9172E9D
:105F240056FD16B86D2F7D2F729555FD16B8E7FDF9
:105F3400672754FD16B8EF77000053FD16B8049098
:105F440052FD16B8502DED9168B9172E56FD16B8AE
:105F54006D2F7D2F729555FD16B8E7FD672754FD0B
:105F640016B8EF77000053FD16B8049052FD16B82A
:105F7400502DED9168B9172E56FD16B86D2F7D2F53
:105F8400729555FD16B8E7FD672754FD16B8EF77EF
:105F9400000053FD16B8049052FD16B8502DED9133
:105FA40068B9172E56FD16B86D2F7D2F729555FDC5
:105FB40016B8E7FD672754FD16B8EF77000053FDC8
:105FC40016B8049052FD16B8502DED9168B9172EED
:105FD40056FD16B86D2F7D2F729555FD16B8E7FD49
:105FE400672754FD16B8EF77000053FD16B80490E8
:105FF40052FD16B8502DED9168B9172E56FD16B8FE
:106004006D2F7D2F729555FD16B8E7FD672754FD5A
:1060140016B8EF77000053FD16B8049052FD16B879
:10602400502DED9168B9172E56FD16B8602F702FBC
:10603400729555FD16B8E7FD672754FD16B8EF773E
:10604400000053FD16B8049052FD16B8502DED9182
:1060540068B9172E56FD16B8602F702F729555FD2E
:1060640016B8E7FD672754FD16B8EF77000053FD17
:1060740016B8049052FD16B8502DED9168B9172E3C
:1060840056FD16B8602F702F729555FD16B8E7FDB2
:10609400672754FD16B8EF77000053FD16B8049037
:1060A40052FD16B8502DED9168B9172E56FD16B84D
:1060B400602F702F729555FD16B8E7FD672754FDC4
:1060C40016B8EF77000053FD16B8049052FD16B8C9
:1060D400502DED9168B9172E56FD16B8602F702F0C
:1060E400729555FD16B8E7FD672754FD16B8EF778E
:1060F400000053FD16B8049052FD16B8502DED91D2
:1061040068B9172E56FD16B8602F702F729555FD7D
:1061140016B8E7FD672754FD16B8EF77000053FD66
:1061240016B8049052FD16B8502DED9168B9172E8B
:1061340056FD16B8612F712F729555FD16B8E7FDFF
:10614400672754FD16B8EF77000053FD16B8049086
:1061540052FD16B8502DED9168B9172E56FD16B89C
:10616400612F712F729555FD16B8E7FD672754FD11
:1061740016B8EF77000053FD16B8049052FD16B818
:10618400502DED9168B9172E56FD16B8612F712F59
:10619400729555FD16B8E7FD672754FD16B8EF77DD
:1061A400000053FD16B8049052FD16B8502DED9121
:1061B40068B9172E56FD16B8612F712F729555FDCB
:1061C40016B8E7FD672754FD16B8EF77000053FDB6
:1061D40016B8049052FD16B8502DED9168B9172EDB
:1061E40056FD16B8612F712F729555FD16B8E7FD4F
:1061F400672754FD16B8EF77000053FD16B80490D6
:1062040052FD16B8502DED9168B9172E56FD16B8EB
:10621400612F712F729555FD16B8E7FD672754FD60
:1062240016B8EF77000053FD16B8049052FD16B867
:10623400502DED9168B9172E56FD16B8612F712FA8
:10624400729555FD16B8E7FD672754FD16B8EF772C
:10625400000053FD16B8049052FD16B8502DED9170
:1062640068B9172E56FD16B8612F712F729555FD1A
:1062740016B8E7FD672754FD16B8EF77000053FD05
:1062840016B8049052FD16B8502DED9168B9172E2A
:1062940056FD16B8622F722F729555FD16B8E7FD9C
:1062A400672754FD16B8EF77000053FD16B8049025
:1062B40052FD16B8502DED9168B9172E56FD16B83B
:1062C400622F722F729555FD16B8E7FD672754FDAE
:1062D40016B8EF77000053FD16B8049052FD16B8B7
:1062E400502DED9168B9172E56FD16B8622F722FF6
:1062F400729555FD16B8E7FD672754FD16B8EF777C
:10630400000053FD16B8049052FD16B8502DED91BF
:1063140068B9172E56FD16B8622F722F729555FD67
:1063240016B8E7FD672754FD16B8EF77000053FD54
:1063340016B8049052FD16B8502DED9168B9172E79
:1063440056FD16B8622F722F729555FD16B8E7FDEB
:10635400672754FD16B8EF77000053FD16B8049074
:1063640052FD16B8502DED9168B9172E56FD16B88A
:10637400622F722F729555FD16B8E7FD672754FDFD
:1063840016B8EF77000053FD16B8049052FD16B806
:10639400502DED9168B9172E56FD16B8622F722F45
:1063A400729555FD16B8E7FD672754FD16B8EF77CB
:1063B400000053FD16B8049052FD16B8502DED910F
:1063C40068B9172E56FD16B8622F722F729555FDB7
:1063D40016B8E7FD672754FD16B8EF77000053FDA4
:1063E40016B8049052FD16B8502DED9128B82F918F
:1063F4001F910F910C94B82CB9CAA82DA530E0F3C5
:10640400A0911401B0911501EAE8F4E0C0911A01D9
:10641400D3E0CD9FE00DF11D7F936EE17EE1CBE1F2
:10642400D1E05881507F452F4295542B588358B959
:1064340052954D914F7358B95991469F58B95295F9
:10644400EF01000058B9C00DD11D599158B95295AA
:106454007A950000000058B9599149F7000058B9DD
:10646400529560911B01000058B959917F9158B918
:106474005295F0911A01F39558B90000000068B9DB
:10648400FA3029F4FF27A0931401B0931501F09377
:106494001A010C94B82C6ACAA82DA530E0F3A09177
:1064A4001401B0911501ED01E2EBF2E0CE0FDF1F14
:1064B400F7E0E0911A01E395E0FBE695FE0F7F9388
:1064C4004F92EEE14E2E6991ED91E7F95081762FCE
:1064D4007295762757FD672768B9ED91E7F956FD60
:1064E40076B90080000055FD76B96991162E54FDE9
:1064F40076B91294162653FD76B907FC61254A94A1
:1065040052FD76B9502D712D39F760911B0168B990
:106514004F907F91EE91F0911A01F395FA3029F49E
:10652400FF27A0931401B0931501F0931A010C9462
:10653400B82CAAEBA4B9AFEFA5B9A0EFA7B9A0E016
:10654400A8B9A0E0A1B9AFEFA2B9A0EFAAB9AFEF83
:10655400ABB9F299539AF2995B98A6B1AC70ABBD02
:10656400B2ECB0938000B9E1B0938100F4E0A2FFF3
:10657400F4E0F0938700FEEFA2FFF6EFF0938600BD
:1065840020928900F4E5F0938800F4E0F0938B0006
:10659400F8EDF0938A00A6E0A0936F00A2E0A4BDFA
:1065A400A1E0A5BDA1E3A7BDA3E8A093B000A1E02D
:1065B400A093B100A0E8A093B3002092B60020926B
:1065C400C000A0E1A093C100A6E6A093C200A2E08F
:1065D400A093C8002092C9000E947678F59909C05A
:1065E400A6E083D7A8E1A093C900A6E0A093CA00BF
:1065F400539A0E942C3BA5E188D0C4E1D1E0A8EDD8
:10660400A993A1E0A993AEE12992AA95E9F7AAEA90
:10661400A0932A01A0932C01209236012092190103
:10662400AEE3A09329010F9320924A010BEE05C01B
:106634000F9308E000934A0109EE00933C010F9187
:10664400089530914A013770373031F4E894F0916D
:10665400F010E1E1F7FF09953A2FA03021F0A430C2
:1066640031F40E947A3BCCE3DEE2ABEE32C0A130DF
:1066740049F420920001A0EEA0930101C8EAD4E7F6
:10668400ADEE27C0A23069F4C0E0D1E02882A0E4D6
:10669400A983A0EAAA83A0EEAB83C8E7DCE4ABEE4F
:1066A40018C0A33059F4AA27BB2744D0A395B395A7
:1066B400B031D9F7ADEEC4E5DAE30BC0A53091F4FF
:1066C400C0E8D0E4A0E2A0930001A0EEA0930101F1
:1066D400A8EBC0935001D0935101A0933C01309397
:1066E4004A010895A63031F40E94473BCCE3DEE230
:1066F400ABEEEFCF0F01F091F010F7FD04C06894FA
:10670400E1E10995E6CF85E00895BF93AF93BA2FF1
:10671400B878B695B695B695AA0FAE7EAB2BA09376
:106724003801AF91BF910895A09336010895A093C5
:1067340019010895DF93CF93AF93AF70A295AA0F79
:1067440008F4A061D1E0CB2FCF70A883AF91CF9193
:10675400DF910895BF93AF93AF70A295AA0F08F489
:10676400A061A295B0913801B07FD8CFAF93A29524
:10677400A7FBAA0FA4F9A07FA0931B01AF910895D2
:10678400488340914A0143FD08954770463081F0A3
:10679400CF93DF935F935CE3C50FD21D46E7C40F2D
:1067A40042E0D41F4091380148835F91DF91CF913B
:1067B40008954F935F936F93AF93BF9340E2592F24
:1067C4005370523061F0533009F44BE2B7FF05C007
:1067D400A095B095A30DB21D4DE20E94DF34592F50
:1067E4005C70692F6073E8944FE24395A051B742FF
:1067F400E0F7A05FB84D5C3009F42BD04FE243952D
:10680400A85EB340E0F7A851BC4F53FD22D06033DB
:1068140009F4D0D04FE24395A456B209E0F7AC593D
:10682400BF4F503009F015D0603209F4C3D04FE2A5
:106834004395AA50E8F70DD0A65F603109F4BAD0A9
:1068440040E34A0FBAD0BF91AF916F915F914F91DE
:106854000895403311F06894B0C091FDAEC0F6F3D2
:1068640090FF0895A9C008954F9390FF05C04B2F42
:10687400429509D04B2F07D04A2F429504D04A2F76
:1068840002D04F9108954F70405D4A3308F0495F3C
:1068940094C00E94010240914A01403009F1443001
:1068A400F9F0D1E0C8EDA7E1463019F0473061F1C5
:1068B400ACE5BEE12992BA95E9F7AA95D1F7413042
:1068C40069F4A0913801DBE0CCE5B0EAA993A9937F
:1068D400BA95E1F7AA24BB24209237010C94FA015B
:1068E40040E2D1E0C8EDA7E1BEE14993BA95E9F7EA
:1068F400AA95D1F740913801A7E1BEE14993BA9531
:10690400E9F7AA95D1F7E6CFF091F010E2E1099505
:10691400E1CF20923701BF91AF910895A730C9F715
:10692400BF91AF91FF93EF93F091F010E6E10995D9
:10693400EF91FF910895AF93BF9320923701A091F7
:106944003601A030A9F4A0914A01A03039F7A7E19B
:10695400AA24B394AB15E9F6ABB5A7FD06C0AA27E4
:10696400B6E1BB2ECF93DF9382C0A22CB22CD1CF41
:10697400A13021F4BF91AF910C942E3AA23049F486
:106984004DE0F699AAD44AE0F799A7D4BF91AF9104
:106994000895A33019F4BF91AF910895A43021F460
:1069A400BF91AF910C94393ABF91AF915AE00E94D4
:1069B400004008954CE201C040E2AF93BF93A09120
:1069C4003701A395A0933701A0913601A53030F08B
:1069D400BF91AF91542F0E9400400895A030D9F088
:1069E400A33059F4A42FBB275F936F930E94DB1C41
:1069F4006F915F91BF91AF910895BF91A0913601BE
:106A0400A13019F4AF910C94423AA230AF9109F439
:106A140064C40C94503AEF93E0914A01E770E0307B
:106A240079F0E43069F0E63059F0E73041F4FF934F
:106A3400F091F010E3E10995FF91EF91DBCF98C05D
:106A4400EF91CF93DF932AD496FD33C099DEA395BB
:106A5400AE3131F4AA27B395B73111F4B6E106C0CB
:106A64005D01DF91CF91BF91AF9108955D01D1E0B8
:106A7400C8ED4F93A6E1BEE14E8D4993BA95E1F777
:106A8400AA95C9F7AEE140E24993AA95E9F7D4E0A3
:106A9400CAE8A6E1BEE14E8D4993BA95E1F7AA95FD
:106AA400C9F7AEE1409138014993AA95E9F74F91AE
:106AB400D8CFAB31B0F6B231A0F6AD5FAA2EEF93CA
:106AC400FF934F925F926F927F9270F85F93E42FDF
:106AD400F6EFB5E04424552466245527A491A7FD78
:106AE400539550FB40F8A6FD539550FB41F8A5FD86
:106AF400539550FB50F8A4FD539550FB51F8A3FD5A
:106B0400539550FB60F8A2FD539550FB61F8F39543
:106B14005527A491A7FD539550FB42F8A6FD539524
:106B240050FB43F8A5FD539550FB52F8A4FD539533
:106B340050FB53F8A3FD539550FB62F8A2FD539507
:106B440050FB63F8F395442D1BDE2196452D18DE8A
:106B54002196462D15DE6C96BA9509F0BBCF5F9150
:106B640070FA7F906F905F904F90FF91EF9179CF83
:106B7400FF93CF93DF936F937F93E42F6091190179
:106B840060FD1DC0F6EFD501DAE0C49136D0B395AF
:106B9400AA2D96FD32D096FDB395F395AA2DDA95DC
:106BA400A1F7AA2DAA5F96FDAA5FAA2E7F916F91E5
:106BB400DF91CF91FF91EF91BF91AF910895FEE8DE
:106BC400EF77AE2FE0E0EA0FF21DAA0FEA0FF21DF5
:106BD400D501D6E0C49155D0B395AA2D96FD51D0D8
:106BE40096FDB395D0FD3196AA2DDA9599F7AA2D85
:106BF400AC5F96FDAC5FAA2ED9CF609138016F933C
:106C04006295C7FD629560933801ABD0A39596FD5C
:106C1400A8D096FDA395C6FD629560933801A1D0D6
:106C2400A39596FD9ED096FDA395C5FD62956093B0
:106C3400380197D0A39596FD94D096FDA395C4FDF5
:106C44006295609338018DD0A39596FD8AD096FD08
:106C5400A395C3FD62956093380183D0A39596FDF7
:106C640080D096FDA395C2FD62956093380179D0DA
:106C7400A39596FD76D096FDA3956F916093380108
:106C8400089560913801D0FDC295762FC7FF7295A3
:106C94007093380166D0A39596FD63D096FDA395B5
:106CA400762FC6FF7295709338015BD0A39596FD3D
:106CB40058D096FDA395762FC5FF72957093380131
:106CC40050D0A39596FD4DD096FDA395762FC4FF85
:106CD40072957093380145D0A39596FD42D096FDE8
:106CE400A3956093380108954F934591403011F472
:106CF4004F91089562DEF9CFFF91EF91EE0FFF1FE0
:106D0400AF93BF93B591BF3F11F0A5910ED0BF9142
:106D1400AF914F934591403031F44F913197F695AF
:106D2400E7953196099449DEF5CFEF93E0914A0156
:106D3400E03071F0E73049F4FF93F091F010E4E1B2
:106D4400F7FF0995FF91EF910895EF915D01089583
:106D5400EF91AE3108F0ADE1B73108F0B6E15D0175
:106D640008950F9300914A0107300F9151F4FF9356
:106D7400EF93F091F010E5E1F7FF0995EF91FF91A2
:106D840008950E941102D1E0C8ED609150016A1784
:106D940028F0609151016B1708F002C00C940C02AA
:106DA40070914A01773069F0753031F0743041F0F8
:106DB400737039F0723008F43AC009F476C091C0A7
:106DC400A9C051E0AC3348F5BE3238F5B0FD550FDB
:106DD400B0FD550FA0FD550FB695A6956EE1B69F73
:106DE400CA0FD21DC00DD11DA2EBB2E0CA0FDB1F2A
:106DF400A881B0913801BF70B295A07FBA1779F01D
:106E0400B0913801BF70AB2BA883A2EBB2E0CA1BD0
:106E1400DB0BB881B52BBF70B8830C940C02A2EBCA
:106E2400B2E0CA1BDB0BB8815095B523F4CF6A2FAF
:106E34006770639540E00894441F6A95E9F7A69546
:106E4400A695A695EA2F65E1F0914A01F2FD60E16D
:106E5400B69FCA0FD21DC00DD11DA0913801F2FFFB
:106E640008C0A695A170E9F44095A881A423A8833D
:106E7400D4CF5E2FB695B695B695F5E1FB9FECE5BC
:106E8400FBE0E00DF11DE50FF21DA0913801AF709C
:106E9400508152955F705A1739F35081507F5A2BA5
:106EA4005083A881A42BA883B8CF6A2F50913801AE
:106EB4005695537043E0637031F0440F440F550FFF
:106EC400550F6A95C9F74095A695A6956EE1B69FAC
:106ED400CA0FD21DC00DD11DA881A423A52BA88340
:106EE4009CCF6A2F509138015F70569508F4586012
:106EF4004FE0617011F0429552954095A6956AE273
:106F0400B69FCA0FD21DC00DD11DA881A423A52BE5
:106F1400A88383CF51E0AC33D0F4BE32C0F4B0FDCB
:106F2400550FB0FD550FA0FD550FB695A6956EE112
:106F3400B69FD1E0C8EDCA0FD21DC00DD11DB091CE
:106F44003801B27029F0B881B52BBF70B88365CF12
:106F5400B8815095B523F9CFCE3108F0CDE1EE31AB
:106F640008F0EDE1D73108F0D6E1F73108F0F6E1A9
:106F7400EC1718F40E2EEC2FC02DFD1718F40F2E5D
:106F8400FD2FD02D0895EC1718F40E2EEC2FC02DE4
:106F9400FD1718F40F2EFD2FD02D08950E94110215
:106FA400DBDF3F0140914A01403051F0443041F071
:106FB4004130C9F5ACE5BBE0F0E875E160E106C03D
:106FC400AAE8B4E0E8EDF1E07EE167E1C71758F51F
:106FD400671648F5D61738F5761628F56C2F7D9F79
:106FE400A00DB11DAC0FB21DE00DF11DEC0FF21D93
:106FF4000090380140E2572F5A955C0F56196C2FB8
:107004001EF0F7FF419302C00C9002940D92661596
:1070140011F06395F5CFA50FB21DE50FF21DD7153D
:1070240011F0D395ECCF0C940C020E9401025F93F3
:10703400AADFAC2FBD2F95DEA395AE17E1F791DE45
:10704400B395FB17E1F78DDEAA95AC17E1F789DE5E
:10705400BA95BD17E1F75F910C94FA010E94010201
:107064005F9391DFBD2FAC2F7CDEAE1711F0A3959B
:10707400FBCF77DEFB1711F0B395F5CF5F910C943E
:10708400FA010E941102E89489DF66DF4C2FBD2FBC
:10709400AC2F05D152EF599351EFA395AE1711F0D0
:1070A4005993FBCF53EF5993A42FB395BF1739F0DE
:1070B400F6D050EF5993AE2FF2D05993F5CFA42FB9
:1070C400EED054EF599351EFA395AE1711F05993A5
:1070D400FBCF55EF59930C940C02D3DF0E9411029D
:1070E4003BDF5E2F5C1B515057FF09F40BC0FBEFD5
:1070F400ECEE0AD0D395FDEFEFE006D0D395FEEE8B
:10710400EDEE02D00C940C02DE010FDE4F2F55DCA5
:10711400652F4E2F52DC6A95E1F74F2F43954DCCE6
:107124000E941102DE014FEFCE1B10F44195C19570
:107134005FEFDF1B10F45195D195CD1760F000C0BF
:107144006C2F66950EDEAE1789F0A40F6D1BD0F779
:10715400B50F6C0FF7CF6D2F669503DEBF1731F0B7
:10716400B50F6C1BD0F7A40F6D0FF7CF0C940C0266
:10717400AF93A0EFA815F1F3A815F1F7AF91089517
:107184000E940102F091F210F7FD03C0E3E20995B9
:1071940019C0A0932801FBE8A6FDFCE8F0933B018D
:1071A400AF73AA0FFDE8E0E8EA0FF21DA591A093E2
:1071B4002601A591A0932701209229012092240160
:1071C400209225010C94FA0120922301409123017D
:1071D4004030E1F398C008954F934091220140302C
:1071E400E1F74F9108955AD0A2EBCA0FA2E0DA1F3B
:1071F400A881BA2FB29520922301409123014030F7
:1072040041F440911C014B3110F4A883F6CFB883AC
:10721400F4CFA88378D042C03F933DED55D020925F
:107224002301409120014470431749F0403021F478
:107234000E943E08342F03C00E945F08342F4091FF
:107244002301403061F440911C014B3120F448810A
:107254004F774883E6CF488140684883E2CF58811E
:107264005F7758833F910895D1E0C3EECA0FD21DD2
:107274002092230140912301403061F440911C018C
:107284004B3120F448814F774883F4CF48814068DC
:107294004883F0CF58815F7758830895D5010F92C2
:1072A4001F92DEE1BD9FD1E0C8EDCA0FD21DC00D13
:1072B400D11D1F900F900895F2DF0F9302EBC00FC2
:1072C40002E0D01F0F910895D3E2BD9FD2E0C4E441
:1072D400CA0FD21DC00DD11D0895FF930E943C1CFE
:1072E40016F086E20EC0FFEFF1B900001A99FECF46
:1072F40042B9F4E6FA95F1F72998F4E6FA95F1F72C
:10730400299AFF9108954F934091390141FD0BC093
:107314004F910895FF91EF91DF91CF91BF91AF917C
:107324004F9144270895AF93BF93CF93DF93EF9387
:10733400FF934D7F40933901A0914A014A2F74D0A5
:1073440040911B016ED040914C016BD0C0E0D1E064
:10735400B0E14991429568D0BA95D9F77DD0C8ED8E
:10736400D1E0A03031F4FEE2EEE165D0FA95E1F728
:10737400D1CFA830D1F4F3E0E3E25DD0FA95E1F7A0
:10738400E3E2F0913A01EF9FC00DD11DF0E1E3E299
:107394004881429549D049914F7746D0EA95C1F743
:1073A4000E942E3AFA9599F7B5CFA13031F4F3E85B
:1073B400E5E141D0FA95E1F7ADCFA23031F4F4E53F
:1073C400EEE139D0FA95E1F7A5CFA33031F4FAE331
:1073D400EAE231D0FA95E1F79DCFA43011F4F7E554
:1073E400C3CFA53031F4F0E4E0E125D0FA95E1F71C
:1073F40091CFA630A1F3A73099F4EEE0F4EE4491D6
:10740400429512D0459110D0449142950DD04591AA
:107414000BD00E942E3AFCE5EEE10DD0FA95E1F78F
:1074240079CF4295469547704F70405D4A3308F0D6
:10743400495F0C94423A48814295F6DF4991F4DF62
:10744400EA95C9F70C942E3ABF93B2E0A03009F044
:10745400B064B4BDBF910895F09B09C04F934DE053
:10746400F69910D04AE0F7990DD04F9108954F93B3
:107474004DE0F69913D04AE0F79910D04F91089552
:10748400F09B0CC0BF93B0913101B030E1F7409351
:107494003201BA95B0933101BF910895F29B0895DA
:1074A4005F935091C80055FFFCCF4093CE005F918D
:1074B4000895F09B10C0BF93B0913301B030E1F751
:1074C400BA95B0933301B0913301B030E1F74091F4
:1074D4003401BF9108954427F29B08954091C80058
:1074E40047FFFCCF4091CE000895F29B08950E947F
:1074F4000102EAE3F5E7B0FD7096BA2FBB0FBE7048
:10750400EB0FF21DB591B093CD00B591B093CC00C3
:10751400B091CA00B670A4FBB3F9A5FF04C0B06271
:10752400A6FBB4F902C0A6FDBB7FA7FDBD7FB09347
:10753400CA000C94FA010823041102080103008113
:1075440000500040002A0823041102080103823479
:10755400411A208C1045F09B17C0BF93B0913301A2
:10756400B030E1F7BA95B0933301409122014D3E1A
:1075740041F0B0913301B030C1F740913401BF9173
:1075840008954BE1BF9108954427F29B08954091DB
:1075940022014D3EB1F34091C80047FFF8CF40911E
:1075A400CE0008950E9401022F930F017E9624912C
:1075B400CEE1D7E0E0E2F6E72BD020922301F00100
:1075C400A2DECCE6D4E020FF04C0B0912001B2FDDD
:1075D400B0961ED040912301403089F3A1E04D3E86
:1075E40079F0A2E0413F61F0A3E0423F49F0A4E01A
:1075F400433F31F0A5E0443F19F021FD06C0DFCF41
:10760400B0912001B2FDAB5F4A2F2F910C94FA0187
:10761400BEE1A591A993BA95E1F708954E4E4E4E59
:107624004E4EC0C0C0C0C0C08080808080802E2EDE
:107634002E2E2E2E6E6E6E6E6E6E0E940102CCE6A3
:10764400D4E0E6DFCEE1D7E0E0E2F6E7E1DF0C9458
:10765400FA01BEB3ACE5B3FDAFE5ACBD2DBCA1E111
:10766400A093B800A0E0B4FFA1E0A093B900A3E008
:10767400B0916B00B0FDA6E038CFA82DA815F1F3AA
:10768400A0912C01B0912B0108950E941102A8ED44
:10769400B1E0C2EBD2E02D922197E9F740E050E04F
:1076A4000FD043954034D9F70C940C0267FF05C002
:1076B4004F934C2FCD2FD42F4F917C2B660F0895D1
:1076C400E0E0F6EFF50FE40F6491C0913801DC2F90
:1076D400D295C07FD07FE3E07727E8DF7295E6DFBD
:1076E40072957D93EA95C1F753955A3049F70895F9
:1076F4000E9401024F93A0E8B7E0E0E0F6EFCAE091
:10770400D0E845914D93DA95E1F7F096F096B0966E
:10771400CA95B1F74F910C94FA01FF93EF93BF70A0
:10772400EFE0FDE8EB1BF491FF0FFA95F0935201A3
:1077340016F4F0935301EF91FF910895AF93ABB515
:10774400A062ABBDAF910895AF93ABB5AF7DF9CF58
:107754000E941102AAE8B4E04EE15F73459FA00DB8
:10776400B11D009038016093380155270E94623B97
:10777400009238010C940C020E941102E42FF6EFDF
:10778400A0E8B7E05F77A50F5AE060E844914C9316
:10779400F395A60FB21D5A95C9F70C940C020E94DA
:1077A40011024F925F926F927F922F93C6E4D1E0C1
:1077B4002C8148A05F846E84798859A16889A22F9E
:1077C400A370E52F660FEE0FA33031F0660FEE0FB6
:1077D400A23011F0660FEE0FF62FA0915801A130E0
:1077E40071F4E2013ED0803011F08FE133C0E30147
:1077F40038D0803011F080E22DC05CD02BC0A23094
:1078040091F4E2012ED0803011F08FE123C0E30126
:1078140037D0803011F082E11DC0ACE3BDE06A0EC8
:107824007B1E6CD017C0A33011F085E113C0A52DC9
:10783400A33010F082E10EC0ACE3BDE04A0E5B1E43
:10784400F20151916191E3010CD0803011F080E29A
:1078540001C05ED02F917F906F905F904F900C94F9
:107864000C02CE0F10F48FE10895A0915001CA17B5
:10787400D0F7DF0FC0F3B0915101DB17A0F70895E3
:10788400659FC00DD11D2296D33008F082E1089582
:10789400A22F5091670160915601E52F660FEE0FFC
:1078A400A33031F0660FEE0FA23011F0660FEE0F29
:1078B400F62F0895571478F0D20134D0E8E8F1E0B7
:1078C40064D0D3012FD0E8E8F1E084D053947394CA
:1078D4006A9591F70895560E760E5A947A94D201C9
:1078E40021D0E8E8F1E051D0D3011CD0E8E8F1E080
:1078F40071D05A947A946A9591F70895F30151934B
:107904006193D2010FD041D053946A95D1F7089571
:10791400F20151916191D30105D05CD073946A95C1
:10792400D1F708956F93C8EDD1E0213011F465E1EA
:1079340003C0253069F460E1B69FC00DD11D6A2FE4
:10794400669566956695C60FD21D4A2F6F91089568
:10795400223069F46EE1B69FC00DD11D6A2F669581
:107964006695C60FD21D4A2F440F6F9108956AE29F
:10797400B69FC00DD11D6A2F66956695C60FD21DA0
:107984004A2F440F440F6F9108957F936F93BF93D1
:10799400AF93652F742F777029F4A991A1936A95F9
:1079A400E1F73FC0B0E8713019F0B6957A95FBCF96
:1079B4007727A991AB9F703019F0A291A029A193C8
:1079C400119273957617A9F7A991AB9FA291A0295B
:1079D400A19327C07F936F93BF93AF93652F742FA9
:1079E400777029F4A191A9936A95E1F71AC00F93CE
:1079F4001F930FEF11E0000F110F7A95E1F7652F38
:107A04007881009570230095A191A19F072A09927E
:107A1400712D6A95C9F768816023672B69930F916B
:107A24001F91AF91BF916F917F9108950E940102C0
:107A34002E013F013FDF0C94FA010E9401022E0146
:107A44003F015CDF0C94FA010E9401022E013F0108
:107A54005FDF0C94FA010E94110250E060E0FAE842
:107A6400EE27C0916701CF77D0915601DF7744911B
:107A74004C9FA12DE0954491E0954D9FB12DA51704
:107A840029F4B61719F4E39591F718C05A2F6B2F00
:107A9400A0916601B0915501A50FB60F0E94B336AF
:107AA400B61BB61B0E94B336A51BA51B0E94B3369A
:107AB400B60FB60F0E94B336E395C9F60C940C02C8
:107AC4000E9411026FEFFAE8EE27C0916701CF77A9
:107AD400D0915601DF7744914C9FA12DE0954491BC
:107AE400E0954D9FB12DB61719F4E395A1F7E6CFB4
:107AF4005A2F6B2FA0916601B09155017A2FB61BB6
:107B0400A51B750F0E94B336B60FB60F0E94B3368D
:107B1400B61BB61BA3957A17A8F7E395E1F6CECF6B
:107B2400409138014F93FF93EF9374D00E947E36B7
:107B34000B0920505245535320454E5445522000C2
:107B4400EF91FF914F91409338013EDB4A3EE9F7B4
:107B540043CBFF91EF910ED0EF93FF936894E0DF56
:107B64000E94F91E0895FF91EF9104D0EF93FF93C3
:107B7400E894D6CFEE0FFF1FC8E8D1E045914993B2
:107B840058E145914993403011F05A95D1F7299223
:107B94003197F695E7953196C8E8D1E0089540917C
:107BA40038014F93FF93EF9335D00E947E360B0834
:107BB400202859296573202F20284E296F20000082
:107BC400EF91FF914F914093380106DB16D004DB0F
:107BD40044270EF443950895FF91EF91CBDFEF9383
:107BE400FF936894DCDF0E94F91E0895FF91EF91E2
:107BF400C1DFEF93FF93E894D2CFE894E5DA4A3EED
:107C040039F04D3E31F04F7D4E3419F04935A9F726
:107C140068940895FF93EF9392E020923601A9911E
:107C24000E948733DF93CF9316F40E94D61EC2E0DE
:107C3400D8E0EBE1FCE00E944338A3E0B9E00E9405
:107C44009736CF91DF9158E14991403051F0DF935D
:107C5400CF935F930E94DF345F91CF91DF915A9568
:107C640099F740913801429540933801EF91FF9183
:107C740008950F931F932F933F93A0935401B093B0
:107C84005701C0936601D093550105D03F912F91C0
:107C94001F910F9108950E940102B6D00E3118F47D
:107CA400173108F415D0A0915401B0915701C09137
:107CB4006601D0915501B983AA83AE3138F4B73146
:107CC40028F435D07370713009F06BD00C94FA013C
:107CD4009BD0239F310F2596C00DD11DC00DD11D02
:107CE400412FE8EDF1E05EE1549FE00DF11DE00F5E
:107CF400F21D522F699161935A95E1F74395431709
:107D040081F740914A01463089F0412FEAE8F4E0D6
:107D14005EE1549FE00DF11DE00FF21D522F6991B9
:107D240061935A95E1F74395431781F708956CD011
:107D3400239F310F2596C00DD11DC00DD11D77276E
:107D4400412FE8EDF1E05EE1549FE00DF11DE00FFD
:107D5400F21D522F619169936F7009F071E05A9589
:107D6400C9F74395431769F7E0916601F09155010E
:107D74004081742B708340914A01463089F0412F31
:107D8400EAE8F4E05EE1549FE00DF11DE00FF21D1E
:107D9400522F619169935A95E1F74395431781F7FF
:107DA400089532D0310F2596412FE8EDF1E05EE1E0
:107DB400549FE00DF11DE00FF21D522F6991619364
:107DC4005A95E1F74395431781F740914A014630AC
:107DD400D1F0412FEAE8F4E05EE1549FE00DF11D9B
:107DE400E00FF21D522F6991660F38F464FB60F9BD
:107DF4006F70462E6081607F642961935A9599F76C
:107E04004395431739F70895C0916601D091550100
:107E14000A8119812C813B8108950E941102E0910D
:107E24003801437001F5A6E1B2E0C4E3D2E0F22DDB
:107E34000BD0A0914A01A63031F0A8ECB4E0C6EE14
:107E4400D4E0FE2F01D06DC062E15AE149914D9317
:107E54005A95E1F7149624966A95B9F75AE1FD9379
:107E64005A95E9F708954130E9F4ACE4B4E0CBE481
:107E7400D4E0F22D0BD0A0914A01A63031F0AEEF40
:107E8400B6E0CDEFD6E0FE2F01D04BC063E159E15F
:107E94004A914E935A95E1F7FE93149725976A9564
:107EA400B1F70895423001F5ACE4B4E0CEE2D4E099
:107EB400F22D0BD0A0914A01A63031F0AEEFB6E01E
:107EC400C0EED6E0FE2F01D02CC062E15AE14A9107
:107ED4004E935A95E1F7149724976A95B9F75AE1A6
:107EE400FE935A95E9F70895A6E1B2E0C7E1D2E01E
:107EF400F22D0BD0A0914A01A63031F0A8ECB4E0E9
:107F0400C9ECD4E0FE2F01D00CC063E159E14991E2
:107F14004D935A95E1F7FD93259614966A95B1F71A
:107F240008950C940C0268941FC04F935F937F9341
:107F340014DB4B3111F481E018C04430A1F341301B
:107F4400B9F7B9DA642FB7DA4095641711F084E20F
:107F54000CC070E85527AFDA540F49937A95D9F7D6
:107F6400AADA451731F4E89488277F915F914F91FD
:107F7400089589E2FACF4F935F937F9341E082DAC9
:107F8400462F80DA40957EDA70E855274991540FE0
:107F940079DA7A95D9F7452F75DAE7CF0E9401028D
:107FA40020923F01B0933F013092640130925D0111
:107FB400C0935E01C0936001D0935F01D0936101CF
:107FC400E0936201F0936301A0935C01B0933F01DD
:107FD4000C94FA010E940102BA2FF8CFA0913F013C
:107FE40008955E984CE54093B80044E84093BC0083
:107FF40044E94093BC00089544EA0EC05093BB008A
:1080040044E80AC044EC08D05091BB00089544E809
:1080140003D05091BB0008954093BC004091BC0034
:1080240047FFFCCF6091B900687F0895E5DF6830B1
:1080340089F4572F550F5E70506AE0DF683151F4B0
:108044005B2FDCDF683231F45A2FD8DF683211F449
:10805400882708958FE05F915F91CACFE7DFCCDF77
:10806400603169F4572F550F5E70516AC7DF603471
:1080740031F4CDDF683519F411968827B9CF8FE034
:10808400B7CF052ED3DF502DB9DF683219F411961E
:108094008827AECF8FE00895AFDF6830A9F4572F5B
:1080A4005770550F5169AADF603471F4ABDF603546
:1080B40059F4A52FACDF683539F4BB27550FAA1F37
:1080C40008F4B095882794CF8FE092CF8827D830D2
:1080D40020F082E24F914F914FEF0895F7DFF99925
:1080E400FECFD2BDC1BDF89A40B521960895EEDF0A
:1080F4008827F999FDCFD2BDC1BDF89A40B4441682
:1081040011F42196089540BDF894FA9AF99A789456
:10811400F999FECFF89A219608954EBD4DB547FFC3
:10812400FDCF4EB508954F934EEFF7DF4F912C9846
:1081340008952C9A08958827F6DF47EDEEDF44274B
:10814400ECDF2C9A4C7B4432B1F34C31A1F38827F9
:10815400443A19F04C3909F081E108958827EBDF9E
:10816400803021F040E040933C1008954C3911F4E4
:1081740048E0F9CF40E1F7CFF1DF403009F408954A
:10818400440F440F440F440F4A950895AA0FBB1F90
:108194004B2FC3DF4A2FC1DF422DBFDFB695A79512
:1081A4000895803059F44F93C6DF803031F4BBDF3B
:1081B40045E5B3DFEBDF2C9ABEDF4F9108958030A5
:1081C40059F44F93B8DF803031F4ADDF43E5A5DFD8
:1081D400DDDF2C9AB0DF4F910895803051F44F9336
:1081E400AADF803029F49FDF46E897DFCFDF2C9A9F
:1081F4004F9108951196B0933D10A0933E1011979E
:10820400ECCF22D2CEDF48D0E8CF7F93772710D0AF
:108214007F9108957F9371E00BD0D42F72E008D042
:10822400C42F7F9108957F9373E002D07F910895C6
:10823400803099F480DF803081F475DF42ED6DDFAA
:10824400AA0FBB1FA3954B2F68DF4A2F66DF472F6A
:1082540064DFB695A79502D02C9A08955EDF5DDFA2
:108264005CDF5BDF5ACF8030B1F465DF803099F496
:108274005ADF42ED52DFAA0FBB1F4B2F4EDF4A2FAE
:108284004CDF472F440F49DFB695A795E7DFD42F7E
:1082940044DFC42F2C9A08957F9370E010D07F910F
:1082A40008957F9371E04D2F0AD072E04C2FC0DF08
:1082B4007F9108957F9373E0BBDF7F9108958030B1
:1082C400A1F44F9338DF4F91803079F42CDF4F9332
:1082D40047E823DF442721DF41E01FDF472F1DDF6D
:1082E4004F914F931ADF2C9A4F910895803091F457
:1082F40022DF8030D1F717DF4F9347E80EDF4427A2
:108304000CDF40E00ADF472F08DF4F914F9305DF72
:108314002C9A4F9108958030D1F4DF93CF934F93EB
:108324005F9309DF803079F4FEDE47E8F6DE442708
:10833400F4DE4427F2DE40E0F0DE55274991EDDE1D
:108344005A95E1F72C9A5F914F91CF91DF9108955F
:108354008030B1F44F935F93EEDE803079F4E3DE46
:1083640047E8DBDE4427D9DE4427D7DE40E0D5DE0C
:1083740055274FEFD2DE5A95E1F72C9A5F914F9132
:1083840008958030E1F4DF93CF934F935F93D3DE6E
:10839400803089F4C8DE46EDC0DE4427BEDE4427C3
:1083A400BCDE40E0BADE4427B8DE5527B6DE49938A
:1083B4005A95E1F72C9A5F914F91CF91DF910895EF
:1083C400BF93AF93DF93CF934F935F937F93C0DFBC
:1083D4004FE062DF44276EDFAA27BB27FEDE11963B
:1083E4004DEFCA2FCF70C13009F44CEF55DF44274D
:1083F40061DFCC27DD2755DFF0DE1196A03019F4BC
:1084040045EE0E94DF3440913C10B41749F70AC08E
:10841400BF93AF93DF93CF934F935F937F939EDE8E
:10842400403091F47F915F914F91CF91DF91AF9163
:10843400BF910895B42FAA271197F5DEC42FBB2747
:10844400AA27F1DE4C1731F4ACDEEDDE439532DFC2
:10845400C4DEE8CF1196E7DE4C17E1F7F5CFDF93E2
:10846400CF934F939EDE4DEFCA2FCF70C13009F4E6
:108474004CEF12DFCFDE219614DF6ADFAEDE4F91C0
:10848400CF91DF9108950E940102AA27BB27ED0135
:1084940065DE4030A1F0F42FB8DE4C3F41F04D3F93
:1084A40031F04B3A21F04F3018F0403908F421965E
:1084B4001196BF1789F740E0DF1709F441E00C94E7
:1084C400FA010F93BF93AF934F93AA27BB27ED01F4
:1084D400FD0144DE403099F0042F97DE4D3F49F40E
:1084E400DF93CF9397DE4D2FCF91DF914F3F21F054
:1084F40021964C3F09F431961196B01771F74F91BC
:10850400AF91BF910F910895FF93EF93DF93CF93B2
:108514004F932F9323DE4030A9F0AA27BB2775DEA3
:10852400242FB0913D10A0913E1040911401B41736
:1085340010F0A2E0BB27FD0168DE4D3F51F46ADE76
:10854400D21738F42F914F91CF91DF91EF91FF9192
:108554000895159640913C10B41709F4BB27BF1732
:1085640059F7AE1749F7AA27BB271BDE4EDE4F3F4C
:1085740031F0405F242F90DE30DEDF01DDCFAFEF3E
:10858400BFEFE0CF4093780150937A0160937C0170
:1085940008950E941102E2DD403019F481E10C9447
:1085A4000C0252D0B41710F08BE1F9CF2EDE4C3F01
:1085B40011F087E1F4CF40917A01403011F48BE15E
:1085C400EECF413810F08BE1EACF7BDFD03021F4DD
:1085D400C41710F488E1E3CFCCE3DFE050E06FEFA1
:1085E40069935A95E9F7B4DE1196B0933D10A093C0
:1085F4003E1040917A01CCE3DFE04F9385DFB993DD
:10860400A9934BEA49DEDF93CF9304DE219649DE3A
:10861400CF91DF9108DE4EDEEDDDFADE4F914A9513
:1086240061F712D0CCE3DFE076DE40917C0134DEEA
:10863400DF93CF93EFDD219634DECF91DF91F3DD2D
:1086440039DECBDDACCF9EDFA0917801A295BA2FA5
:10865400A07FBF70119608950E9411027727F4DF5E
:10866400D4DD4C3F69F0FFDDDF3F49F0BF93AF93AA
:10867400DE01F5DEAF91BF91CBDE7F5FA1F7EFDEC8
:108684000C940C020E9411022F93AA27BB2753DDDE
:10869400BCDD242FD9DFB9DD4C3F21F489E12F91D2
:1086A4000C940C0270917A01703810F08BE1F7CFC2
:1086B400DADDDF3F11F48BE1F2CFDE01CCE3DDE064
:1086C40040917C01413009F4D395423009F4DE5FD6
:1086D40022DEDF93CF939EDDD21759F02196E1DDA0
:1086E400CF91DF9192DDD8DD9EDDE4DD76DD90DE95
:1086F400D6CFB5DE09DF8EDD2196D3DDCF91DF91B4
:108704004BEACADD90DDD6DD68DDED019DDF49DD94
:1087140070917A01770F4D2FE9DD73954C2FE6DDCB
:1087240074DDBADD80DDC6DD58DDB9CF0E941102EB
:108734008BDF6BDD4C3F19F48EE10C940C027091CD
:108744007A01703810F08BE1F8CF8DDDDF3F11F442
:108754008BE1F3CFDE0125DDCCE3DDE040917C014C
:10876400413009F4D395423009F4DE5F0ADEE5CFE7
:108774000E9401024F935F937F9366DF46DD4C3F77
:1087840011F48EE1DACF77276EDDDE0170E0E8E8E0
:10879400F1E069DDD193C19373957032D1F7CDCFF8
:1087A4000004080D11161A1F23282C3035393D42B8
:1087B400464A4F53575B5F64686C7074787C7F8360
:1087C400878B8F92969A9DA1A4A7ABAEB1B5B8BB87
:1087D400BEC1C4C6C9CCCFD1D4D6D9DBDDDFE2E477
:1087E400E6E8E9EBEDEEF0F2F3F4F6F7F8F9FAFB6C
:1087F400FCFCFDFEFEFFFFFFFFFFFFFF00F900F59D
:10880400F3F1F2FC00FAF8F6F4EB5E00F700000076
:10881400007131000000797361773200006378647D
:10882400653433000020766674723500006E626829
:10883400677A360000006D6A75373800002C6B6962
:108844006F303900002E2D6C00705C0000000000B9
:10885400002700000000EA2B00230000003C000079
:108864000000EC000031003437000000302C3235B9
:108874003638EDC3FB2B332D2A39C40000F900F53B
:10888400F3F1F2FC00FAF8F6F4EB0000F700000054
:10889400005121000000595341572200004358441D
:1088A400452440000020564654522500004E4248BC
:1088B400475A260000004D4A552F2800003B4B49DB
:1088C4004F3D2900003A5F4C00503F00000000007B
:1088D400006000000000EA2A00270000003E0000BB
:1088E4000000EC00003100343700000030E932357C
:1088F4003638EDC3FB2B332D2A39C4004400000065
:108904000000000000000000000000000000000063
:108914000000000000000000000000000000000053
:108924000000000000000000000000000000000043
:10893400000000C000000000000000C100000000B2
:108944000000000000002F000000000000000000F4
:10895400000000000000EA000000C2000000000067
:108964000000000000E100E2E0000000E8E9E500AA
:10897400E3E4EDC3FB2BE72D2AE6C4004500000029
:1089840000000000000000000000000000000000E3
:108994000040000000000000000000000000000093
:1089A40000000000000000000000000000000000C3
:1089B4000000000000000000007B5B0000000000DD
:1089C400007D5D000000000000005C00000000006D
:1089D400000000000000007E00000000007C000099
:1089E4000000000000E100E2E0000000EFEEE5001E
:1089F400E3E4EDC3FB2BE72D2AE6C400FFFFFFFFF2
:108A0400FFFFFFFFFFFFFFFEFEFEFEFEFEFEFDFD7D
:108A1400FDFDFDFCFCFCFCFBFBFBFBFAFAFAF9F99F
:108A2400F9F8F8F8F7F7F6F6F6F5F5F4F4F3F3F2E7
:108A3400F2F2F1F0F0EFEFEEEEEDEDECEBEBEAEA53
:108A4400E9E8E8E7E6E6E5E4E4E3E2E1E1E0DFDEE5
:108A5400DEDDDCDBDADAD9D8D7D6D5D4D4D3D2D19B
:108A6400D0CFCECDCCCBCAC9C9C8C7C6C5C4C3C272
:108A7400C1BFBEBDBCBBBAB9B8B7B6B5B4B2B1B06C
:108A8400AFAEADACAAA9A8A7A6A5A3A2A1A09E9D7E
:108A94009C9B99989796949392918F8E8D8B8A89AB
:108AA4008786858382817F7E7D7B7A7877767473EF
:108AB40071706F6D6C6A696766656362605F5D5C47
:108AC4005A595756545351504E4D4B4A48474544B2
:108AD40042413F3E3C3B393836353332302E2D2B24
:108AE4002A2827252422201F1D1C1A1917161412A0
:108AF400110F0E0C0B090706040301000C11161AC2
:108B04001E2225282B2D2F31323333343434343480
:108B1400343434343535363738393B3C3E404345BC
:108B240047494B4D4F51525354545454545351503C
:108B34004E4C4A4745423F3D3A3836343231302F65
:108B44002E2E2E2F303132333536383A3C3E4042C9
:108B5400444647494A4B4D4E4E4F5050505050504A
:108B640050504F4E4D4C4B49484643413E3B3733A2
:108B74002F2B27221D18130D0802FDF8F3EEE9E54B
:108B8400E1DDDAD7D4D2D0CECDCCCCCBCBCBCBCBD2
:108B9400CBCBCBCBCACAC9C8C7C6C4C3C1BFBCBA76
:108BA400B8B6B4B2B0AEADACABABABABABACAEAFD6
:108BB400B1B3B5B8BABDC0C2C5C7C9CBCDCECFD08D
:108BC400D1D1D1D0CFCECDCCCAC9C7C5C3C1BFBD09
:108BD400BBB9B8B6B5B4B2B1B1B0AFAFAFAFAFAF68
:108BE400AFAFB0B1B2B3B4B6B7B9BCBEC1C4C8CCF0
:108BF400D0D4D8DDE2E7ECF2F7FD0207000A141D39
:108C0400272F383F464B50545759595958565450AA
:108C14004C48433E39332E2925201C1916141211B1
:108C2400111112131517191C1F2225272A2C2E3057
:108C34003132323232312F2D2B2825221F1C1916A6
:108C440013110F0D0C0B0A0A0A0B0C0E101214163A
:108C5400181A1C1E1F2020201F1E1C1916120D0876
:108C640003FDF7F0EAE3DDD6D1CBC6C2BFBDBBBA84
:108C7400BBBCBEC2C6CBD1D7DFE6EFF700081019E4
:108C840020282E34393D414344454442403D393443
:108C94002E29221C150F0802FCF7F2EDE9E6E3E1A8
:108CA400E0DFDFDFE0E1E3E5E7E9EBEDEFF1F3F44B
:108CB400F5F5F5F4F3F2F0EEECE9E6E3E0DDDAD70E
:108CC400D4D2D0CECDCDCDCDCECFD1D3D5D8DADD83
:108CD400E0E3E6E8EAECEDEEEEEEEDEBE9E6E3DF09
:108CE400DAD6D1CCC6C1BCB7B3AFABA9A7A6A6A6EA
:108CF400A8ABAFB4B9C0C7D0D8E2EBF58067534294
:108D0400352B221C16120E0C090706050400000060
:108D1400000000000000000000000000807E7B795D
:108D2400777572706E6C6A68666463615F5D5C5AC5
:108D34005857555352504F4D4C4B4948474544435F
:108D440041403F3E3D3C3B3938373635343332328F
:108D540031302F2E2D2C2B2B2A2928282726252568
:108D640024232322222120201F1F1E1D1D1C1C1B07
:108D74001B1A1A19191818181717160089009100C8
:108D84009A00A300AD00B700C200CE00DA00E700ED
:108D9400F400030112012301340146015A016E015A
:108DA40084019B01B301CD01E901060225024502BC
:108DB40068028C02B302DC020803360367039B03D8
:108DC400D2030C0449048B04D00419056705B905C2
:108DD40010066C06CE063507A30717089308150975
:108DE4009F09320ACD0A720B200CD80C9C0D6B0E15
:108DF400460F2F1025112A123F136414000000CCD3
:108E0400C000333000FFF000000CCCCCCCCC333CA1
:108E1400CCFFFCCC000333CCC333333333FFF33305
:108E2400000FFFCCCFFF333FFFFFFFFFA5A5A50633
:108E3400FF604E5440445E4024F42042F24000005F
:108E4400000000000000000000000000000000001E
:108E54000EAE000004E000AAE800EE4E000000445C
:108E64004040AA000066FF666842C4A248A0000011
:108E7400004400004888404222400A4A0004E400BA
:108E840000048000E000000040224880EAAAE04C90
:108E940044E0E2E8E0E2E2E0AAE220E8E2E0E8EA34
:108EA400E0E24880EAEAE0EAE2E004040004048044
:108EB4002484200E0E00842480C268E400EEE04A7C
:108EC400AEA0CACAC0688860CAAAC0E8C8E0E8C838
:108ED4008068EA60AAEAA0E444E0E22A60AC8CA0DC
:108EE4008888E0AEAAA0CAAAA04AAA40EAE8804AB2
:108EF400AA60EAECA068E2C0E44440AAAAE0AAAAF4
:108F040040AAAEA0AA4AA0AA4440E248E064446051
:108F140004A400C444C04A00000000E04400004A25
:108F2400AEA0CACAC0688860CAAAC0E8C8E0E8C8D7
:108F34008068EA60AAEAA0E444E0E22A60AC8CA07B
:108F44008888E0AEAAA0CAAAA04AAA40EAE8804A51
:108F5400AA60EAECA068E2C0E44440AAAAE0AAAA93
:108F640040AAAEA0AA4AA0AA4440E248E024C420F1
:108F74004444448464808842208CEC8041565220CE
:108F8400436869704261736963322056312E353209
:0A8F940000005245563A206120000B
:1090000020202020202020202020202042FFFFFFA1
:10901000FFFFFFFFFFFFFFFFFFFFFFFFFFFFFFFF60
:109C000020202020202020202020202042FFFFFF95
:109C1000FFFFFFFFFFFFFFFFFFFFFFFFFFFFFFFF54
:10A8000020202020202020202020202042FFFFFF89
:10A81000FFFFFFFFFFFFFFFFFFFFFFFFFFFFFFFF48
:10B4000020202020202020202020202042FFFFFF7D
:10B41000FFFFFFFFFFFFFFFFFFFFFFFFFFFFFFFF3C
:10C0000053657269616C4C6F616465724CEAFFFF45
:10C0100000E6E70000E8E900312E3531FFFFFFFFC1
:10C02000E8E0F0E04591423021F445914E3009F4CA
:10C0300001C008950E944B340E947E360000436880
:10C0400069704261736963322073657269616C2043
:10C050006C6F616465722056312E353100000E948C
:10C060007E360200747279696E6720746F20636F88
:10C070006E6E656374207669612000000E94767898
:10C080002EB33AB560916B0022FF2160E0EDFAEC2F
:10C0900020FD749660FD3A960E9476363092360105
:10C0A0000E947E36FF0C507265737320737061635B
:10C0B0006520746F207374617274210D0A00F09B07
:10C0C00011C0A0913301A030E1F774E6AA95A093C6
:10C0D00033010E94BA38A0913301A030A1F07A95C3
:10C0E000C1F7089574E64091CE004091C80047FD25
:10C0F00005C00E94BA387A95C1F708954091CE00E4
:10C10000403231F0089540913401403209F00895F1
:10C1100020923601A0E8A09338010E947E360409DF
:10C1200020636F6E6E656374656420003092360123
:10C130000E947E36FF0C2D2D2D2D2D2D2D2D2D2DDC
:10C140002D2D2D2D2D2D2D2D2D2D2D2D2D2D2D2D1F
:10C150002D2D0D0A00000E947E36FF2020436869C5
:10C16000704261736963322053657269616C204C5F
:10C170006F616465720D0A000E947E36FF2D2D2DC1
:10C180002D2D2D2D2D2D2D2D2D2D2D2D2D2D2D2DDF
:10C190002D2D2D2D2D2D2D2D2D0D0A000E947E369D
:10C1A000FF2053203D2053686F77205374617475CE
:10C1B000730D0A000E947E36FF2042203D20426916
:10C1C0006E6172792055706C6F61642028584D4FF4
:10C1D00044454D290D0A00000E947E36FF20542060
:10C1E0003D20546578742055706C6F61642028413F
:10C1F00053434949290D0A000E947E36FF20412001
:10C200003D20536574204175746F73746172740DB1
:10C210000A000E947E36FF2043203D20436F6E6659
:10C2200069672048617264776172650D0A000E9437
:10C230007E36FF2051203D20517569740D0A0000A3
:10C240000E945B3A4335E1F04337D1F04334B1F01B
:10C250004336A1F0423481F0423671F0443569F042
:10C26000443759F0413459F0413649F0413519F01D
:10C27000413709F0E5CF1CC3C1C04EC36DC143C0F7
:10C2800000C00E947E36FF0C2D2D2D2D2D2D2D2D25
:10C290002D2D2D2D2D2D2D2D2D2D2D2D2D2D2D2DCE
:10C2A0002D2D2D2D0D0A00000E947E36FF2020200E
:10C2B000202020202020205374617475730D0A0003
:10C2C0000E947E36FF2D2D2D2D2D2D2D2D2D2D2D2A
:10C2D0002D2D2D2D2D2D2D2D2D2D2D2D2D2D2D2D8E
:10C2E0002D0D0A0099D30E94FA790E947E36FF0D27
:10C2F0000A507265737320616E79206B6579210035
:10C300000E945B3A15CF0E947E36FF0C2D2D2D2DFD
:10C310002D2D2D2D2D2D2D2D2D2D2D2D2D2D2D2D4D
:10C320002D2D2D2D2D2D2D2D0D0A00000E947E3638
:10C33000FF2020202020202020204175746F73745E
:10C340006172740D0A000E947E36FF2D2D2D2D2D59
:10C350002D2D2D2D2D2D2D2D2D2D2D2D2D2D2D2D0D
:10C360002D2D2D2D2D2D2D0D0A0056D30E947E36FC
:10C37000FF0D0A53656C656374204175746F7374A7
:10C380006172742028312E2E372C20303D6F666666
:10C3900029203A000E945B3A0E94423A403269F1F9
:10C3A000403320F3483310F740534770042F0A9569
:10C3B000ECE0F0E91CE0109FF00D14911C34A1F4A6
:10C3C0000E947E36FF0D0A43616E6E6F74206175A8
:10C3D000746F7374617274206C6F61646572202174
:10C3E00021210D0A0000C2CF5AB5429540775F78EF
:10C3F000542B5ABD0E94857886CF9ACE0E947E36F5
:10C40000FF0C2D2D2D2D2D2D2D2D2D2D2D2D2D2DAB
:10C410002D2D2D2D2D2D2D2D2D2D2D2D2D2D0D0A8F
:10C4200000000E947E36FF20202020202020584D32
:10C430006F64656D2055706C6F61640D0A000E9419
:10C440007E36FF2D2D2D2D2D2D2D2D2D2D2D2D2DF0
:10C450002D2D2D2D2D2D2D2D2D2D2D2D2D2D2D0D2C
:10C460000A00DAD20E947E36FF0D0A53656C6563BE
:10C47000742050726F6772616D2028312E2E38291A
:10C48000203A00000E945B3A0E94423A403209F48E
:10C49000B4CF413338F3493328F74153ECE0F0E9A6
:10C4A0001CE0149FF00D14911C34B9F50E947E36E7
:10C4B000FF0D0A4F7665727772697465206C6F6143
:10C4C000646572203F2028792F6E29000E945B3A14
:10C4D0004E3609F493CF4937C9F7942F0E947E3620
:10C4E000FF0C2D2D3E207472616E73666572207391
:10C4F000746172747320696E2031307320001AEFFA
:10C500000E94BA381A95E1F71AEF0E94BA381A95C4
:10C51000E1F72F922F920C94C228942F0E947E361E
:10C52000FF0C2D2D3E207472616E73666572207350
:10C53000746172747320696E2031307320001AEFB9
:10C540000E94BA381A95E1F71AEF0E94BA381A9584
:10C55000E1F70E94C22852CF0E9476782EB33AB5F6
:10C5600060916B0022FF21600E947E36FF0C2D2D12
:10C570002D2D2D2D2D2D2D2D2D2D2D2D2D2D2D2DEB
:10C580002D2D2D2D2D2D2D2D2D2D0D0A00000E9430
:10C590007E36FF20204368697042617369633220F0
:10C5A000436F6E66696775726174696F6E0D0A001C
:10C5B0000E947E36FF2D2D2D2D2D2D2D2D2D2D2D37
:10C5C0002D2D2D2D2D2D2D2D2D2D2D2D2D2D2D2D9B
:10C5D0002D0D0A000E947E36FF28312920536572F6
:10C5E00069616C2073706565643A2000E0EDFAECD7
:10C5F00020FD749660FD3A960E9476360E947E3643
:10C60000FF0D0A2832292049324320737065656482
:10C610002020203A200024FD08C00E947E36FF31F1
:10C620003030206B487A000007C00E947E36FF340D
:10C630003030206B487A00000E947E36FF0D0A28B9
:10C640003329205350492073706565642020203AB7
:10C65000200023FD08C00E947E36FF35204D487A19
:10C660002020000007C00E947E36FF313536206B47
:10C67000487A00000E947E36FF0D0A2834292045A2
:10C680004550524F4D2061646472203A2000432F80
:10C690004770405D0E94DF340E947E36FF0D0A28FD
:10C6A0003529204C696E6520656E64202020203A73
:10C6B0002000722F707C703841F40E947E36FF6F2C
:10C6C0006E6C79204C46000011C0703441F40E9419
:10C6D0007E36FF6F6E6C79204352000007C00E94C7
:10C6E0007E36FF43522B4C46202000000E947E36AF
:10C6F000FF0D0A2836292053657269616C20492F85
:10C700004F20203A200021FD08C00E947E36FF7392
:10C71000696D706C6520200007C00E947E36FF7333
:10C7200074616E64617264000E947E36FF0D0A2897
:10C7300037292053657269616C20496E7075743AAF
:10C74000200025FF06C00E947E36FF5044330000C3
:10C7500005C00E947E36FF50443100000E947E36A4
:10C76000FF0D0A2838292053746F72652026205245
:10C7700065626F6F740D0A000E947E36FF0D0A53CA
:10C78000706163652072657475726E7320746F20BA
:10C790006D61696E206D656E750D0A000E947E36B2
:10C7A000FF0D0A53656C65637420506172616D659D
:10C7B0007465722028312E2E3829203A00000E94FC
:10C7C0005B3A0E94423A403289F1413338F34933AF
:10C7D00028F7483309F42BC0413331F4632560FF57
:10C7E000232522FF2160C0CE423319F400E1202727
:10C7F000BBCE433319F408E02027B6CE443331F4DE
:10C80000032F03950770387F302BAECE453321F4CC
:10C81000205C08F02064A8CE463319F402E02027FB
:10C82000A3CE473319F400E220279ECE81CC2EBB45
:10C830003ABD60936B000E9485780E947E36FF0CA3
:10C840002D2D2D2D2D2D2D2D2D2D2D2D2D2D2D2D18
:10C850002D2D2D2D2D2D2D2D2D2D2D2D0D0A0000A5
:10C860000E947E36FF2020436869704261736963CD
:10C8700032207265626F6F7473206E6F770D0A00DD
:10C880000E947E36FF2D2D2D2D2D2D2D2D2D2D2D64
:10C890002D2D2D2D2D2D2D2D2D2D2D2D2D2D2D2DC8
:10C8A0002D0D0A000E94BA380E94BA380C9400007C
:10C8B0000E947E36FF0C2D2D2D2D2D2D2D2D2D2D55
:10C8C0002D2D2D2D2D2D2D2D2D2D2D2D2D2D2D2D98
:10C8D0002D2D0D0A00000E947E36FF202053657228
:10C8E00069616C204C6F6164657220517569740DCB
:10C8F0000A000E947E36FF2D2D2D2D2D2D2D2D2D44
:10C900002D2D2D2D2D2D2D2D2D2D2D2D2D2D2D2D57
:10C910002D2D2D0D0A0008950E947E36FF0C2D2D21
:10C920002D2D2D2D2D2D2D2D2D2D2D2D2D2D2D2D37
:10C930002D2D2D2D2D2D2D2D2D2D0D0A00000E947C
:10C940007E36FF202020202020205465787420553A
:10C95000706C6F61640D0A000E947E36FF2D2D2DD4
:10C960002D2D2D2D2D2D2D2D2D2D2D2D2D2D2D2DF7
:10C970002D2D2D2D2D2D2D2D2D0D0A004DD00E944C
:10C980007E36FF0D0A53656C6563742050726F67C5
:10C9900072616D2028312E2E3829203A00000E9425
:10C9A0005B3A0E94423A403209F427CD413338F3D2
:10C9B000493328F74153ECE0F0E91CE0149FF00DF7
:10C9C00014911C34A1F40E947E36FF0D0A43616E5F
:10C9D0006E6F74206F7665727772697465206C6F04
:10C9E00061646572202121210D0A0000C8CF4093A7
:10C9F00049010E947E36FF0C2D2D3E2073656E642A
:10CA00002066696C65206E6F77200D0A00000E9419
:10CA10009E080E943C7980CF00E00E947E36FF5045
:10CA2000000041E3400F0E94423A0E947E36FF3AE6
:10CA30002000F0E9E0E01CE0109FF00D45910E941D
:10CA4000423A1A95D9F744914E3441F40E947E3609
:10CA5000FF2042494E415259200012C04C3441F44B
:10CA60000E947E36FF204C4F41444552200008C0B2
:10CA70000E947E36FF20424153494320200000C0DF
:10CA80001AB512951770103041F01A95011729F454
:10CA90000E947E36FF28412900000E947E36FF0D4D
:10CAA0000A000395083009F0B8CF0E947E36FF0DCA
:10CAB0000A53706163652072657475726E732074B9
:10CAC0006F206D61696E206D656E750D0A000895A9
:10CAD0003936303020283229000033386B34202892
:10CAE0003229000031323030202831290000323420
:08CAF00030302028312900003C
:10CC000020202020202020202020202042FFFFFF65
:10CC1000FFFFFFFFFFFFFFFFFFFFFFFFFFFFFFFF24
:10D8000020202020202020202020202042FFFFFF59
:10D81000FFFFFFFFFFFFFFFFFFFFFFFFFFFFFFFF18
:10E4000020202020202020202020202042FFFFFF4D
:10E41000FFFFFFFFFFFFFFFFFFFFFFFFFFFFFFFF0C
:10F000000C940000FF91FFBF1F900F90AF91BF9134
:10F01000CF91DF91EF91FF916F915F914F91189593
:10F02000A0913D01E0913301E03091F0EF3F21F4F8
:10F03000A0FD0EC0EEE30CC0EA95F5EFB491B5FF6C
:10F0400007C0B0913401B695A0FBB7F9B093340175
:10F05000E0933301E0913101E030B1F0EF3F19F47A
:10F06000E0E5AF770DC0EA95F5EFB491B4FF08C0C5
:10F07000B0913201B0FB0894B795A7F9B093320173
:10F08000E0933101A0933D010895A0913D01E091ED
:10F090003301E03091F0EF3F21F4A0FD0EC0ECE72A
:10F0A0000CC0EA95F5EFB491B7FF07C0B0913401F9
:10F0B000B695A0FBB7F9B0933401E0933301E0912A
:10F0C0003101E03009F3EF3F19F4E0E9AF77D8CF31
:10F0D000EA95F5EFB491B6FFD3CFB0913201B0FB12
:10F0E0000894B795A7F9B0933201CACFC7EFD7E01C
:10F0F0007DD1453A99F0219745EA7AD141EE78D110
:10F1000040E076D140E074D109C0C8EFD7E0422F8B
:10F110006FD1432F6DD1462F6BD10895C8EFD7E043
:10F1200065D14B7F4EBB62D14ABD60D140936B002D
:10F13000F298ECECFF27408155EA508350814083E0
:10F14000553A11F4F59BF29A0895FF93EF9304D189
:10F15000E0934001F0934101EF91FF910895E09118
:10F160004001F0914101A0E2A99FE00DF11DB09690
:10F17000C0EBD1E0A0E2B591B993AA95E1F7BFEF5A
:10F18000B993089547B740FDFDCFB7BFE89547B79E
:10F1900040FDFDCF089547B746FF0895B1E1F2DF86
:10F1A000FACF46B342FF089544E046BB830C921C5D
:10F1B00008954E2F407E19F4B3E0E4DFECDFA0E1C8
:10F1C00009901990B1E0DEDF3296AA95C9F7E030D8
:10F1D00009F008953297B5E0D5DFDDDF3296089566
:10F1E000F8944F93BF93AF9330D1B3E0CBDFD3DF2D
:10F1F0003297CCE3DFE0A0E8329609901990B1E0B5
:10F20000C1DFAA95C9F7B5E0BDDFC5DFAF91BF91FA
:10F210004F9178940895E0914001F0914101B097A9
:10F22000ACE0B591B993AA95E1F7ABB5A7FD089508
:10F23000A6EAB2E0CA0FDB1FACE0B0913801B99387
:10F24000AA95E9F70895E0E0F0E9A0E0BCE0492FD5
:10F25000403031F3EA0FFB1F4A95FACF4091490144
:10F260004770AF93ECE0F0E9ACE0A49FF00D45915E
:10F270005591EE50AF910895F8946CD0C0EBD1E069
:10F28000A3EEB1E05CE04D9149935A95E1F742E479
:10F2900049934CE0499352E140E2B9935A95E9F71A
:10F2A000A09787DF9927B3E2B99FA4E4B2E0A00D4D
:10F2B000B11DC8E8D1E050E24D9149935A95E1F76C
:10F2C000299250E24A91403219F428825A95D1F796
:10F2D000C091E301CF3519F4C8E8D1E004C00E9421
:10F2E0001E00C0EBD1E065DF93959F35E1F6789481
:10F2F000089530D0A3EEB1E05CE045914D935A956E
:10F30000E1F77496992750E2A0EBB1E045914D9357
:10F310005A95E1F7A8E8B1E040E253E24D935A95DF
:10F32000E9F7FF93EF939F930E9420009F91EF9145
:10F33000FF91C8E8D1E0B3E2B99FA1E4B2E0A00D2B
:10F34000B11D53E249914D935A95E1F793959F353D
:10F35000D1F608954091490147704295E0ECE49F51
:10F36000E0E0F0E9E00DF11D0895CCE3DFE04CE0D2
:10F3700050E259934A95E9F752E459935FEF43EF0E
:10F3800059934A95E9F7E6DF2BDF3296CCE3DFE0CD
:10F3900040E25FEF59934A95E9F74BE04F9320DF46
:10F3A00032964F914A95D1F778940C94FA79472F79
:10F3B0004770D2DFFF93EF93CDDFAF91BF914CE069
:10F3C0004F93CCE3DFE040E0559159934A95E1F744
:10F3D000FF93EF93FD0104DF3296DF01EF91FF9180
:10F3E0004F914A9569F778940C94FA790C9470408F
:10F3F0000C947940EF93FF93CF93DF930F931F9378
:10F400000F92C0EFD0E108E01FEF19930A95E9F7DA
:10F41000F0E9ECE005910E3469F431960591C0EF06
:10F42000D0E118E0069518F00F2E06940882219678
:10F430001A95C1F7F45FF53E60F30F901F910F919D
:10F44000DF91CF91FF91EF910895CF93DF930F93C9
:10F45000C0EFD0E10FEF088309830A830F91DF919A
:04F46000CF910895AB
:10F50000010101010101210101010101012181012B
:10F510000100002100110101010121D101010101BE
:10F520002101110101010121D1010101012101117B
:10F530000101010121D101010101010111010101BB
:10F540000101D1010101010101110101010101C10B
:10F55000010101010101010101000101C1010101DC
:10F56000010101010101010001C1010101010100CD
:10F57000010101010101410101010101010101003C
:10F58000000000410000000000000000000000003A
:10F59000000000000000000000000000000000006B
:10F5A000000000000000000000000000000000005B
:10F5B000000000000000000000000000000000004B
:10F5C000000000000000000000000000000000003B
:10F5D000000000000000000000000000000000002B
:10F5E000100000000000000000000000000000000B
:10F5F00020000000000000000000000000000000EB
:10F60000009010800090108000901080009010807A
:10F61000FC28288004C0145028282800000000007E
:10F6200000000000000000000000000000000000DA
:10F6300000000000000000000000000000000000CA
:10F6400000000000000000000000000000000000BA
:10F6500000000000000000000000000000000000AA
:10F66000000000000000000000000000000000009A
:10F67000000000000000000000000000000000008A
:10F6800028C004C0000000002088FC34B4000080C2
:10F690006400640064003C3C181818180000000066
:10F6A0000028000008A08080000004C028800024FA
:10F6B00028008000000044288000C004C418000016
:10F6C00000282828280028281818280000000000F2
:10F6D0008090808008A084408080C8A400004C8472
:10F6E00000000000000000008080601800802828D2
:10F6F000280000002828002828282800002CE8904E
:10F700000090108000901080009010800090108079
:10F710007C444480A8A814504844440024000000BD
:10F7200000183C3C185028280C3000000000000055
:10F73000241824400C401440242400000C003024E1
:10F7400024244424444040246424106460646424D9
:10F75000442444244064646464644048604818005D
:10F76000300060000400140060180C6028000000E5
:10F7700000000000300000000000000C1830000005
:10F7800028A004C02800002840847C6C5844A8802D
:10F79000003C003C003C18183C3C3C3C2400403001
:10F7A000182800001090808004C004C028FC287C29
:10F7B00028440C00000044EC8000C004C424000075
:10F7C00000282828286C2828C01828640000000079
:10F7D0008088A41010908440C004C8A400008C80CD
:10F7E000287C008080004084FCF8303000002448F1
:10F7F000280000002828002828282800002CE8C01D
:10F800000090108000901080009010800090108078
:10F81000FC44448080801450444444283C00000050
:10F8200000183C3C20546C181818181800000004EC
:10F830006428640C14603064646428281800186418
:10F84000646464646460606464180C6C605864642C
:10F8500064646464186464646464046060183C00F4
:10F860001800600004003400600000601800000010
:10F8700000000000300000000000001818180018F8
:10F88000449008A06C1C186C4084FC34B444A880DC
:10F8900024002400640000000000000064241830EC
:10F8A0002428282820888080A4A00C60448044401C
:10F8B00028440C40844444800000C0046C2400446C
:10F8C00000282828286C8080C018445440844810A0
:10F8D0008084BCB020888820D834C8A440848C8020
:10F8E0002C7C00C4C4448080C0082830008020885C
:10F8F000280000002828002828282800002CE8A03C
:10F900000090108000901080009010800090108077
:10F910007C808080808010908480804424186424BF
:10F9200000183C40780C7830300C7C180000000C3B
:10F93000681804183C44600C6464282830400C04A7
:10F94000046464606460606064180C78607C546473
:10F9500064646460186464643C640C60301864001F
:10F960000C2444242C2430207428146C185C742437
:10F970004824742448646464646440181818300C83
:10F98000448810906C34286C80807CD8EC6C6C803F
:10F990006424642464642424242424286060184893
:10F9A000404444442088408490A00C6044FC286477
:10F9B00080440C40844444280000C0046C2400802F
:10F9C00028444444446C80806018C44C600C18186F
:10F9D0008080BC1040848820E82CC8A480804C849F
:10F9E000EC2400C4EC448080C008144800802088C7
:10F9F000280000002828002828282800002CE8E4F7
:10FA00000090108000901080009010800090108076
:10FA1000FC808080B098109080ECEC44003C6464E2
:10FA20000018003C24183000300C2440004000181E
:10FA30007C180C0C6C044418242000006000040C9A
:10FA40002C6444606444447040180C50607C7C64B6
:10FA50004464442418646464183C18601818000056
:10FA6000000464606864486454180C78187C54641A
:10FA70006C6C5460306464643C640C30180C7C80A2
:10FA8000808410906C4040488080FC6CB46C6C802A
:10FA900064046464646464046404181824241830DE
:10FAA0001880442840844084808418308080282432
:10FAB00000440C40844444440000C00428241880BE
:10FAC0008080844080A800006018C480A008402482
:10FAD000A4B0BC4080808080E82CC8A488104084FA
:10FAE000E42428C4EC44D480C00814848080208896
:10FAF000288020882088808020888020882CE8F03A
:10FB00000000000090909090101010108080808075
:10FB10007C8080801090B098408080440040646475
:10FB2000001800401C307800300C7C182800003091
:10FB300054181804400464186404282830400C1831
:10FB40007C4064606460606464180C78606468641D
:10FB5000607C780418643C7C3C1830600C18000011
:10FB6000002064606440306464180C50187C646445
:10FB70006C6C602430646464182C181818180C0C11
:10FB800080842088C430286C80807CD8EC6C6C80A9
:10FB90004020646464646420642018180404183CE1
:10FBA00018008044408440848080301880FC801895
:10FBB00044448040844444440000C0042800244459
:10FBC0008080844080A800443018C480A00824406D
:10FBD000BCD0A41084404084E82CC8A44C8480800D
:10FBE000482428C4EC44F880C0081484808020880D
:10FBF000288020882088808020888020882CE82801
:10FC00000000000090909090101010108080808074
:10FC1000FC8080801090808084C4A8440000643CF4
:10FC20000000003C44686C00181818181800286080
:10FC3000641830640C646430640C281818001800D0
:10FC40007C6464646460606464186C6C60646464A4
:10FC500060686C6418643C7C641860600418000080
:10FC6000006464646460302064180C781864646410
:10FC7000482460043C683C7C3C0830181818001884
:10FC8000448820888018186C8080FC34B46C6C80A8
:10FC900064646464646840644064181864441818B8
:10FCA000400080804084208880843018DC80284098
:10FCB00000446040844444280000C0046C0024C414
:10FCC00044444444446C80443018C44C600C1818BC
:10FCD000BCB0808084402088E44CC4C44C848080C4
:10FCE000282400C4EC44D4D0FCF8148480002828D4
:10FCF000280028280000280028282820882CE83000
:10FD00000000000090909090101010108080808073
:10FD10007C4480441450808044EC442800004458C3
:10FD20000018003C18082C000C300000300028009F
:10FD3000242440240C242430242800300C003018C3
:10FD4000246444244440602464242864406464247B
:10FD5000602C642418241824641840480448004087
:10FD6000002044242424300464246C6C246464241F
:10FD7000600C6044182C183C6404400C18300000DF
:10FD8000449040842800004840847C6C58A84480FB
:10FD900064202424242C64206420242424000000D3
:10FDA000240080288080208890A0600CDCFC44180F
:10FDB00028446040844444EC0000C0046C002400EB
:10FDC00028002828286C804418184454408410487F
:10FDD000BCB0808080801090D094C0048C8040841F
:10FDE000284000C4C444FCF880802884800028286F
:10FDF000280028280000280028282820882CE830FF
:10FE00000000000090909090101010108080808072
:10FE1000FC4480441450A8A84080440000006000C6
:10FE200000000000000000000000000000000000D2
:10FE300000000000000000000000000000000000C2
:10FE400000000000000000000000000000000000B2
:10FE500000000000000000000000000000000000A2
:10FE60000000000000000024000028000000000046
:10FE700060080000000000000024000000000000F6
:10FE800028A08080000000604084FC34ECA84480FE
:10FE90000000000000000000000000001818181802
:10FEA0001800444480801090A4A0C004DC806C3C06
:10FEB00000446000004400800080C004C4002400AE
:10FEC00028002828286C282818182864000000001A
:10FED000A4B08080844008A0C8A480808C800000EA
:10FEE000444000808000D4F8408430480000282836
:10FEF000280028280000280028282824482CE8006A
:10FF00000000000090909090101010108080808071
:10FF10007C2880281450109080EC28000000C0003D
:10FF200000000000000000000000000000000000D1
:10FF300000000000000000000000000000000000C1
:10FF400000000000000000000000000000000000B1
:10FF500000000000000000000000000000000000A1
:10FF60000000000000000000000000000000000091
:10FF70000000000000000000000000000000000081
:10FF800028C080800000000020887CD858000080B5
:10FF900000000000000000000000000030303030A1
:10FFA00000004480808008A004C0C0048CFCA858D5
:10FFB00000006000004400280080C004C40000006D
:10FFC00028002828280028281818280000000000E9
:10FFD0008080000084400000C8A400004824000085
:10FFE00000000000000080800000600080002828E1
:10FFF000280028280000280028282828282CE80085
:00000001FF
